:020000040000FA
:061000004FEF4CF012005E
:0610080028EF08F01200C1
:0610180036EF22F0120089
:06102A00030052990000D2
:10103000E70400000900000050990000FA050000D4
:1010400002000000D2980000800200007E00000034
:10105000DACFE4FFE9CFE4FFEACFE4FFF3CFE4FF28
:10106000F4CFE4FFE652F294D6CFC4F18A0E010128
:10107000C425D66E09B28C820080050E855D3FE1E5
:10108000045004E15F0E831486118C6E09A408D00D
:10109000010E021403E1010E031402E044EC1FF000
:1010A00002A012D0D0EC20F021AE0ED0219E868D71
:1010B0004AEC1FF009A404D02A2A2B222C222D222C
:1010C000FDEC1EF001E1029003A011D0D9EC20F05C
:1010D00025AE0DD0259E8CEC1FF009A404D0322A39
:1010E00033223422352259EC1FF001E10390010E26
:1010F000021451E1010E031401E18BD04CD0060E15
:10110000855D4BE109A408D0010E021403E1010E34
:10111000031402E044EC1FF002A01BD0DAEC1DF037
:1011200021AE17D07F0E2114216E868D4AEC1FF060
:1011300009A404D02A2A2B222C222D228FAF03D0DF
:10114000868F8C8E02D0869F8C9EFDEC1EF001E176
:10115000029003A01AD0ECEC1DF025AE16D07F0E45
:101160002514256E8CEC1FF009A404D0322A3322FA
:101170003422352293AF03D0868B8C8A02D0869B93
:101180008C9A59EC1FF001E10390010E021403E167
:10119000010E03143EE000903CD0070E855D39E15E
:1011A00002A037D009A402D044EC1FF000904AEC12
:1011B0001FF0FDEC1EF001E10290DAEC1DF021AE13
:1011C00012D07F0E2114216E868D09A405D02A2A03
:1011D000000E2B222C222D228FAF03D0868F8C8ED7
:1011E00002D0869F8C9EECEC1DF025AE12D07F0EB7
:1011F0002514256E868909A405D0322A000E3322D3
:101200003422352293AF03D0868B8C8A02D0869B02
:101210008C9A500E86154EE0045005E10F0E831493
:1012200086118C6E0ED086AF02D08B8401D08B9449
:1012300086AB02D0898401D0899486BD8B8C86B917
:10124000898A86AD19D086AF0CD01606000E175AC3
:10125000185A195A09A410D02E062F5A305A315A4A
:101260000BD0162A000E17221822192209A404D026
:101270002E2A2F223022312286A919D086AB0CD0FB
:101280001A06000E1B5A1C5A1D5A09A410D0360605
:10129000375A385A395A0BD01A2A000E1B221C22F0
:1012A0001D2209A404D0362A372238223922AF0E53
:1012B0008617E4D0020E855D58E105A03AD0AF054F
:1012C0000A6EAD51AE111AE1F6EC1EF0EF500001BE
:1012D000EA6A9C25E96E9D51EA22EF6A1CEC21F036
:1012E000EE6AED6A22EC21F0EE6AED6AF6EC1EF091
:1012F000EF6A2FEC21F0EE6AED6A1BD01CEC21F0B6
:10130000B0C1EEFFB1C1EDFF22EC21F0ADC1EEFFA7
:10131000AEC1EDFFF6EC1EF0ACC1EFFF2FEC21F0FB
:10132000EE50ED1006E12FEC21F0ADC1EEFFAEC1A5
:10133000EDFF0001A6510101AC5D17E10001A051D4
:101340000101AD190CE10001A1510101AE1907E144
:10135000010EB96FB66BC15108E08A9806D0B96B1F
:10136000010EB66FC15101E08A88850502E0000ECA
:1013700001D0010E5A6E020E855D02E0000E01D012
:10138000010E5A100EE05EEC1FF001E177D08707E6
:10139000000E885B895B8A5B5EEC1FF06FE000905B
:1013A0006DD0030E855D2AE18B5123E0B2C15AF066
:1013B000B3C15BF0D8905B325A32D8905B325A326C
:1013C0005A50BB6EBFC15CF0C0C15DF0040ED89036
:1013D0005C365D36E804FBE1300E5C16000E5D16EF
:1013E000CF0EBA1400015C105A6E5DC05BF0E8507D
:1013F00003D0BB6ACF0EBA14BA6E3FD0040E855D1F
:101400003DE18651000823E2045002E18D9001D0B5
:101410008C92860503E18D848D82898C020E865D17
:1014200003E18D848D82899C030E865D03E18D949A
:101430008D82899C040E865D03E18D848D92899C4A
:10144000050E865D09E18D948D92899C05D004502E
:1014500002E18D8001D08C82AC51000806E204507C
:1014600002E18B9207D0899205D0045002E18B8271
:1014700001D0898248EC1EF00E90008009A4FDD0B6
:10148000010E001404E1080E091401E1F6D0050E66
:101490000101855D02E0000E01D0010E5B6E070EBA
:1014A000855D02E0000E01D0010E5A6E060E855DCC
:1014B00002E0000E01D0010E5A105B1001E1DDD0F8
:1014C000098E26C080F127C081F128C082F129C091
:1014D00083F1ADA2FED783C1AEFFADA2FED782C11C
:1014E000AEFFADA2FED781C1AEFFADA2FED780C1D7
:1014F000AEFF2AC080F12BC081F12CC082F12DC03B
:1015000083F1ADA2FED783C1AEFFADA2FED782C1EB
:10151000AEFFADA2FED781C1AEFFADA2FED780C1A6
:10152000AEFF1EC080F11FC081F120C082F121C03A
:1015300083F1ADA2FED783C1AEFFADA2FED782C1BB
:10154000AEFFADA2FED781C1AEFFADA2FED780C176
:10155000AEFF8CC180F18DC181F18EC182F18FC14E
:1015600083F1ADA2FED783C1AEFFADA2FED782C18B
:10157000AEFFADA2FED781C1AEFFADA2FED780C146
:10158000AEFF2EC080F12FC081F130C082F131C09A
:1015900083F1ADA2FED783C1AEFFADA2FED782C15B
:1015A000AEFFADA2FED781C1AEFFADA2FED780C116
:1015B000AEFF32C080F133C081F134C082F135C05A
:1015C00083F1ADA2FED783C1AEFFADA2FED782C12B
:1015D000AEFFADA2FED781C1AEFFADA2FED780C1E6
:1015E000AEFF22C080F123C081F124C082F125C06A
:1015F00083F1ADA2FED783C1AEFFADA2FED782C1FB
:10160000AEFFADA2FED781C1AEFFADA2FED780C1B5
:10161000AEFF90C180F191C181F192C182F193C17D
:1016200083F1ADA2FED783C1AEFFADA2FED782C1CA
:10163000AEFFADA2FED781C1AEFFADA2FED780C185
:10164000AEFF36C080F137C081F138C082F139C0B9
:1016500083F1ADA2FED783C1AEFFADA2FED782C19A
:10166000AEFFADA2FED781C1AEFFADA2FED780C155
:10167000AEFFADA2FED70A0EAE6E0C501CE081503C
:101680000B6EE8500D18E81C0C1415E0010E0E143A
:1016900012E10BC0C9F40E80026A036A00800F6A6F
:1016A000106A116A016A200E015C05E2015065ECC6
:1016B0001EF0012AF8D700A013D10101856B0F504D
:1016C00001E1F6D009B28C8006B08C9404019551EA
:1016D00002E0010E956F115002EC1FF0126E050E24
:1016E000125C03E148EC21F005D0060E125C14E117
:1016F000DBEC1FF0BCEC20F00EEC1FF0BCEC20F09B
:10170000040E59EC1DF0EECF98F1EECF99F1EECF2B
:101710009AF1EFCF9BF109D0070E125C11E1DBECDF
:101720001FF0BCEC20F00EEC1FF01EEC22F0EFCF0F
:1017300086F175EC1CF0A2EC1DF0E2EC20F044D038
:10174000020E125C1EE181EC20F01EEC22F0270E4E
:1017500059EC1DF0EECFADF1EDCFAEF1E8EC20F09D
:101760001EEC22F0290E59EC1DF0EFCFAFF11EEC6C
:1017700022F02A0E59EC1DF0EECFB0F1EDCFB1F111
:1017800023D0120403E181EC20F01ED0030E125C82
:101790000EE181EC20F0E2EC20F01EEC22F02C0EA9
:1017A00059EC1DF0EECFB2F1EDCFB3F10DD0040E38
:1017B000125C0AE175EC1CF0EFCF85F11EEC22F013
:1017C000EFCF86F1E8EC20F0070E0101855D02E025
:1017D000000E01D0010E5B6E060E855D02E0000E6C
:1017E00001D0010E5A6E050E855D02E0000E01D09B
:1017F000010E5A105B103AE08BA908D087C11EF089
:1018000088C11FF089C120F08AC121F08BAB08D0BC
:1018100087C122F088C123F089C124F08AC125F054
:101820008BA104D01E6A1F6A206A216A8BA304D090
:10183000226A236A246A256A8BA505D01E681F6860
:1018400020687F0E216E8BA705D02268236824684C
:101850007F0E256EFDEC1EF002E0028001D00290AA
:1018600059EC1FF002E0038001D0039009A414D0CA
:10187000266A276A286A296A2A6A2B6A2C6A2D6ACC
:101880002E6A2F6A306A316A326A336A346A356A7C
:10189000366A376A386A396A115065EC1EF0112AC7
:1018A0001350115C01E3116A0F501AE00F0618D0B3
:1018B000040195050CE10401E80E986F030E996F81
:1018C00096C49AF497C49BF40401020E956F01012B
:1018D000876B886B896B8A6B06B08C8409B28982AE
:1018E00080AE078008A002D081A00780045003E1E9
:1018F0008C9C8C9802D08B9C899A09AE04D0F2946F
:101900008A0ED66E099E09A203D089928C908C9281
:10191000E552E5CFF4FFE5CFF3FFE5CFEAFFE5CFF2
:10192000E9FFE5CFDAFF11000101C56BC66BC76B9C
:10193000C86BB4EC1FF0C3EC1FF0D16BD26BD36B50
:10194000D46BD56BD66BD76BD86BD96BDA6BDB6B83
:10195000DC6BB9EC1FF0E16BE26BE36BE46BE56B06
:10196000E66BE76BE86BE96BEA6BEB6BEC6BBEEF7E
:101970001FF0D9CFE6FFE1CFD9FFE652DF6A020EB2
:10198000DF5C2DE2DF50040DF3CFE9FFF4CFEAFF77
:101990008C0EE926010EEA22010EEE6EEE6AEE6A68
:1019A000EE6ADF50040DF3CFE9FFF4CFEAFF940EA7
:1019B000E926010EEA22EE6AEE6AEE6AEE6ADF506E
:1019C000040DF3CFE9FFF4CFEAFFA40EE926010EE0
:1019D000EA22EE6AEE6AEE6AEE6ADF2AD0D70101E9
:1019E000856B0101866B0101876B886B896B8A6B44
:1019F0000101AD6BAE6B0101AC6B0101AF6B01017D
:101A0000B06BB16B0690096A92809F9C010EE66EE6
:101A1000E66A13EC2EF0E552E552010EE66E0B0E6F
:101A2000E66E13EC2EF0E552E5528D8496948D828D
:101A30009692898C929C8D8096908B8294928C9CAD
:101A4000959C8C9E959E8C9895988C9A959A949E30
:101A5000828E000000000000000000000000000076
:101A60000000000000000000000000000000000076
:101A70000000000000000000948E829E0101010E13
:101A8000C16F05808A989398899692960101010EFC
:101A9000B66F046A0101010EB96FDF6A200EDF5CC8
:101AA00009E2DF50EA6A580FE96E010EEA22EF6A96
:101AB000DF2AF4D70101BA6BBB6BBC6BBD6B076A45
:101AC0000101C36B0101010EC26F0F6A106A116A36
:101AD000010E136E050E146E156A9380F19E088038
:101AE000939681960B6A0C6A0D6A0E90A3EC19F01E
:101AF000D58CD59AD596D594D592D580D66AD58EE3
:101B0000F184F294F28AE552E552E7CFD9FF120050
:101B10004BEC1DF0030E34EC1EF047EC20F0E66AAF
:101B2000D950C0EC20F00401845101E0ABD0DF04B7
:101B300020E132EC21F007E10101010EC16F0590B7
:101B400059EC1EF00ED0D4EC1DF0010EEE1805E19C
:101B5000ED5003E10101C16B03D00101010EC16F22
:101B60000580000EE66EE66AB9C1E6FF50EC1FF094
:101B700087D0020EDF5C2DE132EC21F008E1046A2F
:101B800096909492959C959E9598959A1BD0D4EC9E
:101B90001DF0010EEE180CE1ED500AE1010E6CECA7
:101BA0001FF094949294949C929A9592929268D0F9
:101BB000D4EC1DF0020EEE1863E1ED5061E1020E6F
:101BC0006CEC1FF094849284948C928A9582928219
:101BD00057D0040EDF5C07E1010EDBCFA0F0020E50
:101BE000DBCFA1F04DD0050EDF5C07E1010EDBCFAE
:101BF0009EF0020EDBCF9FF043D0080EDF5C0FE1BA
:101C0000D4EC1DF0080ED880EE54000EED5403E223
:101C1000080E93EC1FF0010EDBCF9AF031D0090EC5
:101C2000DF5C0FE1D4EC1DF0060ED880EE54000E00
:101C3000ED5403E2060E93EC1FF0010EDBCF9BF098
:101C40001FD00A0EDF5C03E19AEC1FF009D00B0EE7
:101C5000DF5C03E19AEC1FF013D00C0EDF5C07E1B0
:101C6000010EDBCFA4F0020EDBCFA5F009D00D0EE4
:101C7000DF5C06E132EC21F002E0088001D0089040
:101C800049EC1DF0030EE15C02E2E16AE55247EF28
:101C90001DF060EC21F0E10EE66E010E05EC20F087
:101CA000E50EE66E010EAFEC21F0D7EC1FF028E157
:101CB0000101C2511DE0D151D211D311D41105E15E
:101CC000D951DA11DB11DC1103E0D0EC1EF010E188
:101CD000E151E211E311E41105E1E951EA11EB11DF
:101CE000EC1103E0D5EC1EF003E10401848D08D073
:101CF000B4EC1FF0B9EC1FF0BEEC1FF0C5EC20F007
:101D000040EF1EF060EC21F06AEC21F0E50EE66E8B
:101D1000010E05EC20F0A9EC21F02EE10101C251E9
:101D200027E0D151D211D311D4110AE1D951DA11DE
:101D3000DB11DC1105E1DD51DE11DF11E01103E003
:101D4000D0EC1EF015E1E151E211E311E4110AE1DA
:101D5000E951EA11EB11EC1105E1DD51DE11DF1162
:101D6000E01103E0D5EC1EF003E10401848D04D002
:101D7000B4EC1FF0C5EC20F040EF1EF04BEC1DF072
:101D8000110EE12612EC20F022EC22F0D950010FC6
:101D900002EC22F0090F2FEC20F06AEC21F0D95070
:101DA000050F02EC22F00D0F2FEC20F02BEC22F0AF
:101DB00059E10101C25106E0DAEC1EF003E1040131
:101DC000848D50D07EEC1EF0D96BDA6BDB6BDC6B54
:101DD000E96BEA6BEB6BEC6B08EC1EF0010EDBCFF2
:101DE000D1F1020EDBCFD2F1030EDBCFD3F1040E23
:101DF000DBCFD4F1050EDBCFE1F1060EDBCFE2F154
:101E0000070EDBCFE3F1080EDBCFE4F1090EDBCFE9
:101E1000D9F10A0EDBCFDAF10B0EDBCFDBF10C0EC2
:101E2000DBCFDCF10D0EDBCFE9F10E0EDBCFEAF1FB
:101E30000F0EDBCFEBF1100EDBCFECF1000E01014A
:101E4000DD6DDE1FDE23DF1FDF23E01FE023ED6DEE
:101E5000EE1FEE23EF1FEF23F01FF023C3EC1FF064
:101E600036EC21F0110EE15C02E2E16AE55247EF47
:101E70001DF073EC21F06AEC21F0A9EC21F00DE1EA
:101E80000101C25106E0DAEC1EF003E10401848D89
:101E900004D07EEC1EF036EC21F040EF1EF073EC27
:101EA00021F0E10EE66E010EAFEC21F0D7EC1FF051
:101EB00011E10101C25106E0DAEC1EF003E1040178
:101EC000848D08D07EEC1EF0B9EC1FF0BEEC1FF044
:101ED00036EC21F040EF1EF04BEC1DF0050EE12634
:101EE000DE6ADE6ADE6ADD6ADD52DD520EB025D2C0
:101EF00009B408D0EBEC1EF005E2030ECD6FCE6BFB
:101F0000CF6BD06BFE0EDB5032E10101800ED81595
:101F100014E0800ED41517E1000EFFEC20F0D16D17
:101F2000D21FD223D31FD323D41FD423D96DDA1FBA
:101F3000DA23DB1FDB23DC1FDC23800EE81517E030
:101F4000800EE41503E00401848DF7D1000E07EC48
:101F500021F0E16DE21FE223E31FE323E41FE4230A
:101F6000E96DEA1FEA23EB1FEB23EC1FEC230101D1
:101F70002A6B2B6B2C6B2D6B2E6BD9C140F0DAC109
:101F800041F0DBC142F0DCC143F0020EABEC1EF0CD
:101F900040500101D15D4E6E4150D2594F6E4250BA
:101FA000D359506E4350D459516EDDC140F0DEC15B
:101FB00041F0DFC142F0E0C143F0060EABEC1EF091
:101FC0004E5040240101D16F4F504120D26F5050EC
:101FD0004220D36F51504320D46FE9C140F0EAC191
:101FE00041F0EBC142F0ECC143F0020EABEC1EF04D
:101FF00040500101E15D4E6E4150E2594F6E42503A
:10200000E359506E4350E459516EEDC140F0EEC1BA
:1020100041F0EFC142F0F0C143F0060EABEC1EF010
:102020004E5040240101E16F4F504120E26F50506B
:102030004220E36F51504320E46F01012F6B09A44C
:1020400016D0FD0EDB500DE12F892F8BCDC12BF16A
:10205000CEC12CF1CFC12DF1D0C12EF10101CD6B3C
:1020600003D00101030ECD6FCE6BCF6BD06BCDC112
:102070004EF0010E17EC1FF03EE0040EDB6AD90EA5
:10208000E96E010EEA6E0101D151EE244E6ED2517D
:10209000EE204F6ED351EE20506ED4513DEC1DF02A
:1020A00002E611EC1EF01DE350EC1DF01CE1DD0E0C
:1020B000E96E010EEA6ED951EE244E6EDA51EE2031
:1020C0004F6EDB51EE20506EDC513DEC1DF002E610
:1020D00011EC1EF006E350EC1DF005E1800EE0155A
:1020E00002E053EC1FF0040EDB5003E001012F85EA
:1020F00002D001012F81CDC14EF0020E17EC1FF06E
:102100003CE0040EDB6AC8EC1FF00101E151EE2453
:102110004E6EE251EE204F6EE351EE20506EE451D0
:102120003DEC1DF002E611EC1EF01DE350EC1DF03D
:102130001CE1ED0EE96E010EEA6EE951EE244E6EE1
:10214000EA51EE204F6EEB51EE20506EEC513DEC1B
:102150001DF002E611EC1EF006E350EC1DF005E167
:10216000800EF01502E053EC1FF0040EDB5003E08C
:1021700001012F8702D001012F83DD0EE96E010ED0
:10218000EA6EEE500101D95DD96FEE50DA59DA6F7F
:10219000EE50DB59DB6FEE50DC59DC6FED0EE96E73
:1021A000010EEA6EEE50E95DE96FEE50EA59EA6F12
:1021B000EE50EB59EB6FEE50EC59EC6F0401C60595
:1021C00002E18D908B92D1C130F1D2C131F1D3C1F6
:1021D00032F1D4C133F1FE0EDB5009E0C9C138F150
:1021E000CAC139F1CBC13AF1CCC13BF102D087EC85
:1021F0001EF0D9C148F1DAC149F1DBC14AF1DCC1B5
:102200004BF1DDC140F1DEC141F1DFC142F1E0C17E
:1022100043F1E1C134F1E2C135F1E3C136F1E4C18A
:1022200037F1FE0EDB5006E001013C6B3D6B3E6B6F
:102230003F6B02D090EC1EF0E9C14CF1EAC14DF1C8
:10224000EBC14EF1ECC14FF1EDC144F1EEC145F1EE
:10225000EFC146F1F0C147F1FE0EDB5003E0010192
:10226000070E02D00101060E296F09AA5AD0F4EC1C
:1022700021F01BEC20F077EC21F04C0E4E6E8B0E13
:1022800059EC1CF048C1E6FF49C1E6FF4AC1E6FF30
:102290004BC1E6FF1BEC20F0470E4E6E8B0E59EC47
:1022A0001CF040C1E6FF41C1E6FF42C1E6FF43C169
:1022B000E6FF1BEC20F0FBEC21F01BEC20F086ECA1
:1022C00021F0380E4E6E8B0E59EC1CF04CC1E6FF1F
:1022D0004DC1E6FF4EC1E6FF4FC1E6FF1BEC20F00B
:1022E000330E4E6E8B0E59EC1CF044C1E6FF45C117
:1022F000E6FF46C1E6FF47C1E6FF1BEC20F02E0ECD
:102300004E6E8B0E59EC1CF02FC14EF04F6A506A86
:10231000516A2FC1E6FFA2EC21F01BEC20F056EC35
:102320001DF009BC0AD013500F5CFDE20EB005D0C1
:1023300079EC1CF001E3106A0F2A050EE15C02E261
:10234000E16AE55247EF1DF077EC20F0D50EE66E1E
:10235000010EC1EC21F0E66EE50EE66E010EFEEC1C
:102360001FF00401845101E012008CDA49EF1DF0E6
:102370004BEC1DF0250EE126DE6ADD6A020EDB6AFB
:10238000030EDB6A040EDB6A050EDB6A060EDB6AEF
:10239000070EDB6A080EDB6A090EDB6A0A0EDB6ACF
:1023A0000B0EDB6A0C0EDB6A0D0EDB6A0E0EDB6AAF
:1023B0000F0EDB6A100EDB6A110EDB6A120EDB6A8F
:1023C000130EDB6A140EDB6A150EDB6A160EDB6A6F
:1023D00094EC0CF0E4EC21F0030E53EC1CF0E66AF4
:1023E000D950020F02EC22F0060F02EC22F00A0F85
:1023F00002EC22F00E0F02EC22F0120F6FEC20F034
:102400000101C25101E184D0120EDB50010802E249
:102410000401848DDECF4EF0DDCF4FF0010E4E5C17
:10242000000E4F5808E3EBEC21F0A80ED880EE54D4
:10243000610EED5402E20401848D020EDBCF41F007
:10244000030EDBCF42F0040EDBCF43F0050EDFECD2
:102450001EF002E6FEEC1DF008E3D950020F38EC46
:102460001EF002E61AEC1EF002E20401848D060E54
:10247000DBCF41F0070EDBCF42F0080EDBCF43F09D
:10248000090EDFEC1EF002E6FEEC1DF008E3D95069
:10249000060F38EC1EF002E61AEC1EF002E2040110
:1024A000848D0A0EDBCF41F00B0EDBCF42F00C0E19
:1024B000DBCF43F00D0EDFEC1EF002E6FEEC1DF06C
:1024C00008E3D9500A0F38EC1EF002E61AEC1EF0B1
:1024D00002E20401848D0E0EDBCF41F00F0EDBCF44
:1024E00042F0100EDBCF43F0110EDFEC1EF002E6DF
:1024F000FEEC1DF008E3D9500E0F38EC1EF002E69A
:102500001AEC1EF002E20401848D0401845144E1BE
:102510000EB042D009AA39D0280E4E6E8B0E59EC5F
:102520001CF0DECF4EF0DDCF4FF00EEC1DF01F0E95
:102530004E6E8B0E59EC1CF0D950020F45EC21F079
:10254000160E4E6E8B0E59EC1CF0D950060F45EC52
:1025500021F00B0E4E6E8B0E59EC1CF0D9500A0F69
:1025600045EC21F0000E4E6E8B0E59EC1CF0D9504C
:102570000E0F45EC21F0F40E4E6E8A0E59EC1CF055
:10258000120EACEC20F056EC1DF0D20E4E6E8A0E00
:1025900039EC21F049EC1DF0250EE15C02E2E16A24
:1025A000E55247EF1DF016EC21F0010EDF6E12EC44
:1025B00020F0010EE66ED90EE66E010EC1EC21F0A0
:1025C000E66EE90EE66E010EC1EC21F00101C95D77
:1025D000000ECA59000ECB59000ECC5904E2010E70
:1025E000C96FCA6B09D0D880A80E74EC1FF006E240
:1025F000A80EC96F610ECA6FCB6BCC6B13500F5C0A
:10260000FDE2DF040AE1F29E01015EEC1FF003E14E
:10261000855101E1DF6AF28EF4D716C040F017C091
:1026200041F018C042F019C043F07CEC1FF00101EA
:10263000D925D56F3D50DA21D66F3E50DB21D76FBB
:102640003F50DC21D86F1AC040F01BC041F01CC0C5
:1026500042F01DC043F07CEC1FF00101E925E56F5D
:102660003D50EA21E66F3E50EB21E76F3F50EC21F1
:10267000E86FC3EC1FF014D849EC1DF040EF1EF0DA
:1026800012EC20F0E66AD50EE66E010E05EC20F0A5
:10269000E50EE66E010EFEEC1FF002D849EF1DF0CC
:1026A000FBEC20F009AA1BD0CC0E4E6E8A0E59EC22
:1026B0001CF0C9C1E6FFCAC1E6FFCBC1E6FFCCC131
:1026C000E6FF1EEC1DF0510E4E6E8B0E59EC1CF009
:1026D0006BEC1EF03D0E4E6E8B0E95EC21F00EB0A5
:1026E000A3D0D880A80E010174EC1FF003E3DAEC4C
:1026F0001EF006E1AC0E4E6E8A0E39EC21F094D03D
:10270000D0EC1EF004E1D5EC1EF001E18DD0CDC17E
:102710002FF120EC1FF002E18D908B920101800ED1
:10272000D81502E0B4EC1EF0800EE81502E0BCEC17
:102730001EF0D50EE96E010EEA6E030EEB50E8199D
:10274000E8AE02D0E83508D0E551EE5CE651EE582F
:10275000E751EE58E851EE582AE387EC1DF029ECDA
:102760001FF00101D5EC1EF01CE089EC20F033ECE9
:102770001DF092EC20F0EDEC1CF004E10101010EE3
:10278000346F11D098EC1DF007E10101346935690F
:1027900036697F0E376F34D0C4EC1EF032EC1FF078
:1027A0002FD00101346B356B366B376B29D087EC3A
:1027B0001DF032EC1FF00101D0EC1EF01CE092EC99
:1027C00020F033EC1DF089EC20F0EDEC1CF004E17E
:1027D0000101010E306F11D098EC1DF007E10101ED
:1027E0003069316932697F0E336F0AD0C4EC1EF054
:1027F00029EC1FF005D00101306B316B326B336B6C
:102800000FEC21F090EC1EF0A1EC1FF009AA02D011
:102810000AEC20F013500F5CFDE20EB005D079EC0D
:102820001CF001E3106A0F2A040EE15C02E2E16A87
:10283000E55247EF1DF077EC20F0D90EE66E010E61
:10284000AFEC21F0C8EC1FF00101D951EE24D56F97
:10285000DA51EE20D66FDB51EE20D76FDC51EE203F
:10286000D86FC8EC1FF0EE50D95DE56FEE50DA5925
:10287000E66FEE50DB59E76FEE50DC59E86F02D897
:1028800049EF1DF0FBEC20F00EB000D109AA1BD0DF
:10289000A20E4E6E8A0E59EC1CF0C5C1E6FFC6C1F1
:1028A000E6FFC7C1E6FFC8C1E6FF1EEC1DF09C0EA7
:1028B0004E6E8A0E59EC1CF06BEC1EF0960E4E6EAE
:1028C0008A0E95EC21F00101C25110E0C551C611EC
:1028D000C711C81102E10401848DEBEC1EF002E285
:1028E0000401848D0401845101E0D0D0CDC12FF1C9
:1028F0000101D0EC1EF031E1D5EC1EF02EE101011A
:10290000010E296FA00E0101C55D860EC659010E8C
:10291000C759000EC85907E3A00EC56F860EC66FD3
:10292000010EC76FC86BC5C12BF1C6C12CF1C7C161
:102930002DF1C8C12EF1190E456E466A476A486AE4
:102940003BEC1FF071EC4BF03CC02BF13DC02CF187
:102950003EC02DF13FC02EF18DD020EC1FF002E1E2
:102960008D908B920101800ED81502E0B4EC1EF020
:10297000800EE81502E0BCEC1EF00A0E4E6ED70E7B
:102980004F6EA30E506E4C0E516E3BEC1FF034ECAC
:1029900020F008EC41F0B1EC20F00101D0EC1EF089
:1029A00027E092EC20F05DEC1DF00BE2C25104E058
:1029B000720E4E6E8A0E3FD0C96BCA6BCB6B800E07
:1029C000CC6FDAEC1EF00BE1C25104E04E0E4E6EFD
:1029D0008A0E31D0010EC96FCA6BCB6BCC6BC9C1EB
:1029E00030F1CAC131F1CBC132F1CCC133F105D0E4
:1029F0000101306B316B326B336B0FEC21F0010155
:102A0000D5EC1EF029E089EC20F05DEC1DF00BE226
:102A1000C25104E02A0E4E6E8A0E0DD0C96BCA6BED
:102A2000CB6B800ECC6FDAEC1EF00DE1C25106E0EC
:102A3000060E4E6E8A0E39EC21F028D0010EC96FB9
:102A4000CA6BCB6BCC6BC9C134F1CAC135F1CBC1F8
:102A500036F1CCC137F105D00101346B356B366BE3
:102A6000376B90EC1EF00101A1EC1FF009AA02D017
:102A70000AEC20F009BC0AD013500F5CFDE20EB046
:102A800005D079EC1CF001E3106A0F2A040EE15C1A
:102A900002E2E16AE55247EF1DF04BEC1DF0030E38
:102AA000A4EC20F0A8EC1FF053EC1CF004018451BE
:102AB0003CE1F29E050E0101855D06E0060E855D96
:102AC00003E0070E855D03E1DE52010EDD6E0F505F
:102AD00003E0DE52010EDD6E856B020EDB6A200E16
:102AE000F36E020EDBCFF4FFF350F45C07E2020E4C
:102AF000DB5065EC1EF0020EDB2AF1D7106A116A7A
:102B00000F6ADF0409E1045003E18D808B8204D059
:102B1000040402E18C828982F28ED4EC21F0C3B1EC
:102B200002D056EC1DF049EC1DF0030EE15C02E210
:102B3000E16AE55247EF1DF0A8EC20F0B9C14EF074
:102B40004F6A506A516A4EAE03D04F685068516860
:102B50004EC0E6FFA2EC21F019EC21F0C3B102D087
:102B600056EC1DF049EF1DF04BEC1DF0030EA4ECEC
:102B700020F08450040B08E18450020B05E18050E2
:102B8000400B02E1010E23D08450040B09E0845075
:102B9000020B06E18050400B03E1020EF36E19D0E8
:102BA0008450040B08E18450020B05E08050400B78
:102BB00002E1040E0CD08450040B08E08450020B98
:102BC00005E08050400B02E1080E01D0100EF36EBC
:102BD000020EF3CFDBFF045008E184B003D0020EF5
:102BE000DB50DF6E82B210D009D004040DE183B255
:102BF00003D0020EDB50DF6E80B206D0020EDB5037
:102C0000E76E010EE7CFDBFFDFCF4EF04F6A29EC16
:102C100020F01EEC1DF042EC1EF0D4EC21F0C3B10C
:102C200002D056EC1DF049EC1DF0030EE15C02E20F
:102C3000E16AE55247EF1DF04BEC1DF0020EE12674
:102C4000DE6ADD6A28EC22F0A8EC1FF0030E53ECDC
:102C50001CF0040184510FE10101B90504E1CDEC40
:102C60001FF0E66A04D0CDEC1FF0010EE66E50ECCA
:102C70001FF049EC1DF0020EE15C02E2E16AE55250
:102C800047EF1DF0F7EC20F0E5EC1EF005EC22F02C
:102C900068EC1FF0030F6FEC20F063EC1FF00401F1
:102CA000845124E1030EDB50070802E2E5EC1EF03C
:102CB000DF50030802E2030EDF6E030EDB50030F4A
:102CC0000001A65D07E059EC1EF0030EDB50030F78
:102CD0000001A66F010EDBCFE6FF020EDBCFE6FFA1
:102CE000DFCFE6FF50EC1FF049EC1DF0050EE15C74
:102CF00002E2E16AE55247EF1DF04BEC1DF0060ED3
:102D0000E126FE0EDB0403E129EC1EF04BD0FE0EA3
:102D1000DB50020805E129EC1EF0040EDB6A44D00A
:102D2000FE0EDB50030834E129EC1EF0040EDB6AD2
:102D3000A0C09EF0A1C09FF0F29E050EDB6A200E9F
:102D4000F36E050EDBCFF4FFF350F45C1FE2050ECB
:102D5000DB5002EC1FF0020816E1050EDB502F0DD0
:102D60004BEC20F011EC22F0EF500001A65D0BE1DE
:102D7000050EDB5068EC1EF0270E59EC1DF0A0C0CC
:102D8000EEFFA1C0EDFF050EDB2AD9D7F28E0CD0E5
:102D90009EC0DEFF9FC0DDFF020EA4C0DBFF030E5E
:102DA000A5C0DBFF53EC1FF08986C2C4BEF4C3C4C8
:102DB000BFF4C4C4C0F4C5C4C1F4040EDBCFE6FF45
:102DC000FC0EDBCFE6FFFD0EDBCFE6FF020EDBCF16
:102DD000E6FF030EDBCFE6FFA6C0E6FFCDEC1FF05B
:102DE00028EC21F0060EE15C02E2E16AE55247EFD1
:102DF0001DF0FBEC20F047EC20F0E76E020EE7CF71
:102E0000DBFF040184512CE1020EDB5029E1E7ECE9
:102E100021F0E76E030EE7CFDBFF0401845120E1D0
:102E2000030EDB501DE109BC19D013500F5CFDE20D
:102E3000105068EC1EF0DFCFEFFFADEC1DF011EC91
:102E400022F0010EDBCFEFFFADEC1DF0040EEF6EB4
:102E5000102A1350105C01E3106A0F2A49EC1DF090
:102E6000040EE15C02E2E16AE55247EF1DF028EC56
:102E700022F0FE0E0101BA5DFF0EBB59FF0EBC59D8
:102E8000FF0EBD5905E2BA2B000EBB23BC23BD23A8
:102E900049EF1DF028EC22F00101BA51BB11BC1121
:102EA000BD1105E0BA07000EBB5BBC5BBD5B49EF23
:102EB0001DF04BEC1DF0050EE126E4EC21F0070EB1
:102EC00053EC1CF063EC1FF0DB500BE1DFCFBAF1E9
:102ED000010EDBCFBBF1020EDBCFBCF1030EDBCF6B
:102EE000BDF149EC1DF0050EE15C02E2E16AE5523C
:102EF00047EF1DF0A8EC20F0BAC1E6FFBBC1E6FF2A
:102F0000BCC1E6FFBDC1E6FF19EC21F0C3B102D0A0
:102F1000B1EC1EF049EF1DF04BEC1DF0020E15EC6C
:102F200022F047EC20F0E7EC21F0040184510DE1A0
:102F3000010EDB501F0803E2DE521F0EDD6E84EC33
:102F40001FF0DFCFEFFF49EC1DF0020EE15C02E263
:102F5000E16AE55247EF1DF04BEC1DF0020EA4ECC8
:102F600020F0E7EC21F00401845116E1010EDB5062
:102F70001F0803E2DE521F0EDD6E84EC1FF0EFCF60
:102F80004EF04F6A29EC20F019EC21F0C3B102D0C9
:102F9000B1EC1EF049EC1DF0020EE15C02E2E16AC8
:102FA000E55247EF1DF0A8EC20F007504E6E4F6A37
:102FB000506A516AE66EA2EC21F019EC21F0C3B11F
:102FC00002D0B1EC1EF007B0079049EF1DF09DBC98
:102FD000FED7A8EC20F000C14EF001C14FF00EEC7E
:102FE0001DF042EC1EF016C14EF017C14FF00EEC72
:102FF0001DF00101C3B102D0B1EC1EF049EF1DF08C
:1030000016EC21F0E0D8DF6EA8EC20F00F0EDF14F4
:10301000DF6E0101B95103E0100EDF10DF6E07A073
:1030200003D0200EDF10DF6E0401945104E0400E47
:10303000DF10DF6E946B0EA003D0800EDF10DF6E0A
:10304000020EE66EDFCF4EF04F6A29EC20F09FECC7
:1030500046F0526E050EE15E5250B1EC1EF007B024
:10306000079040EF1EF0F7EC20F0030EDB6A05EC52
:1030700022F063EC1FF068EC1FF0030F6FEC20F000
:103080000401845101E098D0D4EC1DF0FF0ED880EB
:10309000EE54030EED5405E2010EDB68030ED2EC94
:1030A0001FF0DF50010802E2010EDF6E030EDB505D
:1030B000010802E2E5EC1EF0DF0409E1040EDB503A
:1030C000030805E10101BF6B020EC06F06D0010EBF
:1030D000DBCFBFF1020EDBCFC0F1CAB415D0CB6895
:1030E000FC0ECA140009CA6E9D920F0152815293C0
:1030F000F00EBA140C09BA6E3F0EBA140009BA6E7B
:103100000E010E0ECC6FCA84030EDB502AE1DF5095
:1031100023E0BFC14EF0C0C14FF0D8904F324E32C5
:10312000D8904F324E324E50BB6EBFC150F0C0C12E
:1031300051F0040ED89050365136E804FBE1300EC1
:103140005016000E5116CF0EBA14000150104E6EDC
:1031500051C04FF0E85003D0BB6ACF0EBA14BA6E1C
:1031600029D009BC27D013500F5CFDE2105068EC49
:103170001EF02C0E59EC1DF0BFC1EEFFC0C1EDFFDB
:10318000ADEC1DF0EE52EE52EE6AEE6AEE6AEE6AB9
:10319000ADEC1DF0EE52050E59EC1DF0DFCFEFFF48
:1031A000ADEC1DF0030EEF6E102A1350105C01E31E
:1031B000106A0F2A49EC1DF0050EE15C02E2E16A9B
:1031C000E55247EF1DF04BEC1DF0040E34EC1EF001
:1031D000030EDB6AF29E01015EEC1FF002E0010EBD
:1031E000DF6E855102E0010EDF6E0F5006E0010E2A
:1031F000DF6EF36E030EF3CFDBFFDF5006E0FDEC76
:103200001EF003E0DE52010EDD6EDF5006E059ECE9
:103210001FF003E0010ED2EC1FF0F28E030EDBCFA5
:10322000E6FF020EDB50E8244F6E010EDB50040D6A
:10323000F3CF4EF0DF50080DF3504E104F10E55213
:10324000E7104E6E040EE15C02E2E16AE552E16EC7
:103250004E503DEF21F0F7EC20F0030EDB6AB3DFB8
:1032600063EC1FF0010EE66EE66EF1EC29F0E5521C
:10327000E552040EDBA002D0E5EC1EF0040EDBA24A
:1032800003D0010ED2EC1FF0040EDBA403D0DE52FB
:10329000010EDD6E040EDBA602D0010EDF6EDFCF65
:1032A0004EF04F6A0EEC1DF042EC1EF0010EACEC3D
:1032B00020F042EC1EF0020EACEC20F042EC1EF0CE
:1032C000030EACEC20F056EC1DF0050EE15C02E2C2
:1032D000E16AE55247EF1DF04BEC1DF0080EE126C8
:1032E000A8EC20F0F29E16C0DFFF010E17C0DBFF36
:1032F000020E18C0DBFF030E19C0DBFF040E1AC05C
:10330000DBFF050E1BC0DBFF060E1CC0DBFF070E3C
:103310001DC0DBFFF28ED9CFE9FF23EC1DF042EC9C
:103320001EF0D950040F45EC21F00101C3B102D0C9
:1033300056EC1DF049EC1DF0080EE15C02E2E16A7A
:10334000E55247EF1DF0F29E48EC1EF0F28E12009F
:1033500028EC22F0F8DF49EF1DF0FBEC20F000C371
:10336000DFFF31DB02E063DBFEE101C352F095DAFF
:1033700002E05DDBFEE102C352F08FDA02E057DBD0
:10338000FEE103C352F0A0DA04E3ADA2FED767DB8F
:1033900003D0ADA2FED712DBB8EC1DF004E3ADA262
:1033A000FED75DDB03D0ADA2FED708DBBCEC1DF081
:1033B00004E3ADA2FED753DB03D0ADA2FED7FEDA05
:1033C000C0EC1DF004E3ADA2FED749DB03D0ADA2F3
:1033D000FED7F4DAC4EC1DF004E3ADA2FED73FDB68
:1033E00003D0ADA2FED7EADAC8EC1DF004E3ADA22B
:1033F000FED735DB03D0ADA2FED7E0DACCEC1DF072
:1034000004E3ADA2FED72BDB03D0ADA2FED7D6DA04
:10341000D0EC1DF004E3ADA2FED721DB03D0ADA2BA
:10342000FED7CCDAAE6E000E04C3DFFFCCDA02E0CA
:10343000FEDAFEE105C352F030DA02E0F8DAFEE12E
:1034400006C352F02ADA02E0F2DAFEE107C352F0D4
:103450003BDA04E3ADA2FED702DB03D0ADA2FED778
:10346000ADDA86DB04E3ADA2FED7F9DA03D0ADA274
:10347000FED7A4DA81DB04E3ADA2FED7F0DA03D0F5
:10348000ADA2FED79BDA7CDB04E3ADA2FED7E7DA80
:1034900003D0ADA2FED792DA77DB04E3ADA2FED76C
:1034A000DEDA03D0ADA2FED789DA72DB04E3ADA287
:1034B000FED7D5DA03D0ADA2FED780DA6DDB04E308
:1034C000ADA2FED7CCDA03D0ADA2FED777DA68DBA7
:1034D00004E3ADA2FED7C3DA03D0ADA2FED76EDA05
:1034E000AE6E000E08C3DFFF6EDA02E0A0DAFEE186
:1034F00009C352F0D2D902E09ADAFEE10AC352F0CF
:10350000CCD902E094DAFEE10BC352F0DDD904E33A
:10351000ADA2FED7A4DA03D0ADA2FED74FDA28DBE6
:1035200004E3ADA2FED79BDA03D0ADA2FED746DA04
:1035300023DB04E3ADA2FED792DA03D0ADA2FED71F
:103540003DDA1EDB04E3ADA2FED789DA03D0ADA2DB
:10355000FED734DA19DB04E3ADA2FED780DA03D05C
:10356000ADA2FED72BDA14DB04E3ADA2FED777DAE7
:1035700003D0ADA2FED722DA0FDB04E3ADA2FED763
:103580006EDA03D0ADA2FED719DA0ADB04E3ADA2EE
:10359000FED765DA03D0ADA2FED710DAAE6E000E0C
:1035A0000CC3DFFF10DA02E042DAFEE10DC352F095
:1035B00074D902E03CDAFEE10EC352F06ED902E0AB
:1035C00036DAFEE10FC352F07FD904E3ADA2FED795
:1035D00046DA03D0ADA2FED7F1D9CADA04E3ADA230
:1035E000FED73DDA03D0ADA2FED7E8D9C5DA04E3B1
:1035F000ADA2FED734DA03D0ADA2FED7DFD9C0DA50
:1036000004E3ADA2FED72BDA03D0ADA2FED7D6D904
:10361000BBDA04E3ADA2FED722DA03D0ADA2FED717
:10362000CDD9B6DA04E3ADA2FED719DA03D0ADA244
:10363000FED7C4D9B1DA04E3ADA2FED710DA03D0C5
:10364000ADA2FED7BBD9ACDA04E3ADA2FED707DA50
:1036500003D0ADA2FED7B2D9AE6E000E10C3DFFF0D
:10366000B2D902E0E4D9FEE111C352F016D902E06A
:10367000DED9FEE112C352F010D902E0D8D9FEE142
:1036800013C352F021D904E3ADA2FED7E8D903D089
:10369000ADA2FED793D96CDA04E3ADA2FED7DFD991
:1036A00003D0ADA2FED78AD967DA04E3ADA2FED774
:1036B000D6D903D0ADA2FED781D962DA04E3ADA298
:1036C000FED7CDD903D0ADA2FED778D95DDA04E319
:1036D000ADA2FED7C4D903D0ADA2FED76FD958DAB8
:1036E00004E3ADA2FED7BBD903D0ADA2FED766D905
:1036F00053DA04E3ADA2FED7B2D903D0ADA2FED710
:103700005DD94EDA04E3ADA2FED7A9D903D0ADA2AC
:10371000FED754D9AE6E000E14C3DFFF54D902E0B9
:1037200086D9FEE115C352F0B8D802E080D9FEE197
:1037300016C352F0B2D802E07AD9FEE117C352F0B4
:10374000C3D804E3ADA2FED78AD903D0ADA2FED779
:1037500035D90EDA04E3ADA2FED781D903D0ADA2EC
:10376000FED72CD909DA04E3ADA2FED778D903D06D
:10377000ADA2FED723D904DA04E3ADA2FED76FD9F8
:1037800003D0ADA2FED71AD9FFD904E3ADA2FED76C
:1037900066D903D0ADA2FED711D9FAD904E3ADA200
:1037A000FED75DD903D0ADA2FED708D9F5D904E381
:1037B000ADA2FED754D903D0ADA2FED7FFD8F0D921
:1037C00004E3ADA2FED74BD903D0ADA2FED7F6D805
:1037D000AE6E000E18C3DFFFF6D802E028D9FEE176
:1037E00019C352F05AD802E022D9FEE11AC352F0AE
:1037F00054D802E01CD9FEE11BC352F065D804E3A3
:10380000ADA2FED72CD903D0ADA2FED7D7D8B0D960
:1038100004E3ADA2FED723D903D0ADA2FED7CED804
:10382000ABD904E3ADA2FED71AD903D0ADA2FED71F
:10383000C5D8A6D904E3ADA2FED711D903D0ADA255
:10384000FED7BCD8A1D904E3ADA2FED708D903D0D6
:10385000ADA2FED7B3D89CD904E3ADA2FED7FFD862
:1038600003D0ADA2FED7AAD897D904E3ADA2FED764
:10387000F6D803D0ADA2FED7A1D892D904E3ADA269
:10388000FED7EDD803D0ADA2FED798D8AE6E040E09
:10389000E15C02E2E16AE552FAD052EC20F0CFDBC3
:1038A000080E1F0B1200E66E11EC33F0E552C7EF65
:1038B00021F04F6E506A4EC0E6FFE66E50C0E6FF44
:1038C00082EC46F0C7EF21F0EDDBDFCF80F1010E97
:1038D000DBCF81F1020EDBCF82F1030EDBCF83F170
:1038E000010183390F0B73EF20F011502F0D4BEFB7
:1038F00020F01050F0EC21F029C1EEFF2AC1EEFFBC
:103900002BC1EEFF2CC1EEFF2DC1EEFF2EC1EEFF4D
:103910002FC1EEFF30C1EEFF31C1EEFF32C1EEFF2D
:1039200033C1EEFF34C1EEFF35C1EEFF36C1EEFF0D
:1039300037C1EEFF38C1EEFF39C1EEFF3AC1EEFFED
:103940003BC1EEFF3CC1EEFF3DC1EEFF3EC1EEFFCD
:103950003FC1EEFF40C1EEFF41C1EEFF42C1EEFFAD
:1039600043C1EEFF44C1EEFF45C1EEFF46C1EEFF8D
:1039700047C1EEFF48C1EEFF49C1EEFF4AC1EEFF6D
:103980004BC1EEFF4CC1EEFF4DC1EEFF4EC1EEFF4D
:103990004FC1EEFF50C1EEFF51C1EEFF52C1EEFF2D
:1039A00053C1EEFF54C1EEFF55C1EEFF56C1EEFF0D
:1039B00057C1EEFF102A1350105C1200410E010196
:1039C0008425F60F1200010EDB6A020EDB6A030E7D
:1039D000DB6A35DB080E1F0B1200EFEC40F0ABDBAF
:1039E0006EDB51C049F008EC41F0F8DBAC0E4E6ED6
:1039F000C50E4F6EA70E506E470E516E60DB496EBE
:103A00005BEC41F0EBDB1BDB466A476A800E486EDD
:103A10003F0EC4DB3CEC42F0010A12001ADB1BEF44
:103A200020F0E66AF1EC29F0E552E5521200D89058
:103A30004E364F3650365136E8061200D9EC46F075
:103A4000E552C7EF21F0DACFEAFFEECFE6FFEECF87
:103A5000E6FFEECFE6FFEFCFE6FF1BEF20F0300EE4
:103A6000010184251200EFEC40F065DBDBEC21F076
:103A7000FBDA5BEC41F0B1EF20F0EE20516EB5ECDB
:103A800021F0EBEC21F0D890EB50000A1200E16E2F
:103A9000F4D3E66AF6D3D9CFE6FFE1CFD9FF12001F
:103AA000CEDA4E504F10501051101200020EE66E3A
:103AB000E8D3E926000EEA221200EFEC40F0000EF7
:103AC000DFCF46F0010EDBCF47F0020EDBCF48F030
:103AD000030EDBCF49F05BEC41F0FCEC41F040C061
:103AE000C9F141C0CAF142C0CBF143C0CCF1D8808A
:103AF000000E01014054000E4154000E4254800E4D
:103B000043541200E66E000EDA20E66E1200DBEC83
:103B100021F0EDEC40F00FDBAC0E466EC50E476EAB
:103B2000A70E486E470E496E5BEC41F0FCEF41F08A
:103B300086DA466A476A486A4F0E30DB33EC42F059
:103B4000010A1200EE52EE52EECF87F1EECF88F16D
:103B5000EECF89F1EFCF8AF1120010502F0D4BEF0D
:103B600020F00A50E96EEA6AD890E936EA36120087
:103B7000AE6E0F0E8315B7D2AE6E82390F0BB3D275
:103B8000AE6E0F0E8215AFD2AE6E81390F0BABD277
:103B9000AE6E0F0E8115A7D2AE6E80390F0BA3D279
:103BA000AE6E0F0E80159FD2D950010FE96EDACF9D
:103BB000EAFF12009C51A4279D51A5239E51A623E4
:103BC0009F51A723A4518C27A5518D23A6518E2345
:103BD000A7518F23D0EF20F0A051A827A151A923EE
:103BE000A251AA23A351AB23A8519027A9519123F5
:103BF000AA519223AB519323D9EF20F0D880000E25
:103C00004154800E4254000E4354000E445412009E
:103C1000DFCFE6FF010EE66E6CEC0FF0E552E552E9
:103C20001200000EEE5C000EEE58000EEE58000E74
:103C3000EE581200000EEE5C800EEE58FF0EEE58AD
:103C4000FF0EEE581200E66AD9CFE6FFDACFE6FFA4
:103C50001200A0C0DEFFA1C0DDFF020EA2C0DBFF8C
:103C6000030EA3C0DBFF1200E0DB020EDB6A1200D2
:103C7000E96EDACFEAFFD880030EEB50FF0A12009C
:103C8000E552FBD22C0EE66E83EC26F0E5521200D4
:103C9000166A176A186A196A1A6A1B6A1C6A1D6A08
:103CA0001E6A1F6A206A216A226A236A246A256AB8
:103CB0001200E66A000EE66EE66AE66EE66AA6C0E6
:103CC000E6FFE66EE66A28EF21F08ADBEF6A120073
:103CD00087DBEE521200D5C1E6FFD6C1E6FFD7C1A1
:103CE000E6FFD8C1E6FF1BEF20F0EECF90F1EECF5C
:103CF00091F1EECF92F1EFCF93F11200D56BD66B2D
:103D0000D76BD86BE56BE66BE76BE86B1200D5C140
:103D100038F1D6C139F1D7C13AF1D8C13BF112001F
:103D2000E5C13CF1E6C13DF1E7C13EF1E8C13FF13B
:103D3000120030C1E6FF31C1E6FF32C1E6FF33C1F8
:103D4000E6FF120034C1E6FF35C1E6FF36C1E6FFEB
:103D500037C1E6FF1200456E466A476A486AC8EFF7
:103D600041F0010EE66E8DD2800E01012A112A6FFC
:103D7000000E0101FFEF20F0200E01012A112A6F31
:103D8000000E010107EF21F0DECF41F0DECF42F05F
:103D9000DECF43F0DDCF44F0DD52DD52FCEF41F0E9
:103DA000D551D611D711D8111200E551E611E711FE
:103DB000E8111200C951CA11CB11CC111200DBCF8E
:103DC00044F04434000E44181200010EF36E030E4A
:103DD000F3CFDBFF1200D880030E0101CD55000E9A
:103DE000CE55000ECF55000ED05512000A50EA6A8B
:103DF000710FE96E000EEA2212009451951196118E
:103E000097111200EDDAEF501200EECFA0F1EECFD5
:103E1000A1F1EECFA2F1EFCFA3F11200EECF94F11A
:103E2000EECF95F1EECF96F1EFCF97F112004E164F
:103E30004F6A506A516A4E504F1050105110120084
:103E400001012B6B2C6B2D6B2E6B2A6B0401C605AD
:103E5000120040C030F141C031F142C032F143C0E4
:103E600033F1120040C034F141C035F142C036F1A7
:103E700043C037F11200C5C140F0C6C141F0C7C10F
:103E800042F0C8C143F01200262A000E2722282241
:103E9000292212009407000E955B965B975B120037
:103EA0007DEC16F074D2010EF36E040EF3CFDBFF3F
:103EB0001200985199119A119B1112008751881183
:103EC00089118A111200E76E040EE7CFDBFF1200A2
:103ED000010EE66ED9501200046E96809482958C85
:103EE000958E9588958A1200C955610ECA55000EA7
:103EF000CB55000ECC5512004568466847684868A7
:103F000071EC4BF03C501200010EDB50EA6A580F86
:103F1000E96E010EEA22120086899807000E995B6D
:103F20009A5B9B5B1200F36E010EF3CFDBFF020E78
:103F3000DB6A1200010EDBCFA2F0020EDBCFA3F092
:103F400012004C6B4D6B4E6B4F6B050E296F1200C0
:103F5000010EE66ED9CFE6FFDACFE6FF1200610E62
:103F6000E926000EEA221200C96BCA6BCB6BCC6B40
:103F70001200DD6BDE6BDF6BE06B1200ED6BEE6B46
:103F8000EF6BF06B1200CD6BCE6BCF6BD06B120072
:103F9000E90EE96E010EEA6E1200DECFE6FFDDCF1C
:103FA000E6FF1200F36E020EF3CFDBFF1200DF6EAE
:103FB0000401845112006CD92CDAEECFA4F1EECFBB
:103FC000A5F1EECFA6F1EFCFA7F123DA040E71DD54
:103FD000EECFA8F1EECFA9F1EECFAAF1EFCFABF182
:103FE0001CDAEECF9CF1EECF9DF1EECF9EF1EFCF3C
:103FF0009FF113DA040E5DDD05EF1FF0C2D9E66E06
:10400000CD0EE66E010E1AEF22F0E66E060E4BDCC8
:10401000E66A1200E9D912DD6AD9EDD90FDD76D949
:1040200056EF1DF094EC0CF013DAE66AC90EE66E5A
:10403000010E1AEF22F0F5EC46F0E552A8D1CBD9EB
:10404000EECF4EF0EECF4FF0EECF50F0EFCF51F07D
:104050001200506A516A4EC0E6FFA2EF21F052DD15
:10406000060E21DCE66A1200EDEC40F041C052F091
:1040700042C053F043C054F044C055F041C046F034
:1040800042C047F043C048F044C049F084D19CD9B5
:10409000010E53EF1CF0FA51F324E96EFB51F420AA
:1040A000EA6E1200536A546A556A52504E125350C7
:1040B0004F125450501255505112B5EF21F08BD978
:1040C000EECF41F0EECF42F0EECF43F0EFCF44F031
:1040D0004EC046F04FC047F050C048F0120012DD0D
:1040E000010E53EF1CF0846FE8500908120094ECA5
:1040F0000CF0AED9E66AC50EE66E010E9BD9E66AF3
:10410000120075EC1CF0EFCF85F175EC1CF0A2EFFE
:104110001DF0E5C140F0E6C141F0E7C142F0E8C161
:1041200043F01200D5C140F0D6C141F0D7C142F0F2
:10413000D8C143F0120041C04EF042C04FF043C01E
:1041400050F044C051F0120070D9E66E11EF1DF02E
:10415000010EE66E11EF1DF0DBCF4EF04F6A0EEF51
:104160001DF041C0DEFF42C0DEFF43C0DEFF44C0A1
:10417000DDFFDD52DD52120061D90E0E59EF1DF048
:10418000010FC0DC030E53EF1CF0DFCFE6FFE66A41
:104190006CEC0FF0E552E55249EF1DF0496EFBD093
:1041A0008C511E268D511F228E5120228F5121228B
:1041B0001200905122269151232292512422935190
:1041C000252212003BD9050E74DCEFCF8BF11200D3
:1041D00075EC1CF026D9EFCFACF1120044C0EDFF16
:1041E00043C0EDFF42C0EDFF41C0EFFF120053DCC2
:1041F000050E34EF1EF04FDC040EE1261200D56DE3
:10420000D61FD623D71FD723D81FD8231200E56D7A
:10421000E61FE623E71FE723E81FE823120077DD08
:104220000101486B496B4A6B4B6B120034DCE65260
:10423000120004DC0101120094DC890EE926000E54
:10424000EA2212008EDC790EE926000EEA22120024
:1042500083EC3FF04E6E080EE15E4E50120081DCA2
:10426000AFEF1FF0A1DCEE50ED101200D1DC49EFF2
:104270001DF059EC1CF056EF1DF0E552E7CFD9FFC9
:1042800012000FEC2AF0E5521200E96E23EF1DF048
:1042900075EC1CF0EFCF85F1D1D8060E0ADCEECF1D
:1042A0008CF1EECF8DF1EECF8EF1EFCF8FF1C6D83E
:1042B000060E59EC1DF0040E59EC1DF075EF1EF0C2
:1042C000B5DF94EC0CF0C4D8BDD8D50EE66E010E67
:1042D0009CDEC7D0DD0EE66E010E97DEE10EE66EC7
:1042E000010E05EF20F0A2DF9DDEACD8BAD0510E52
:1042F0004E6E8B0E59EC1CF038C1E6FF39C1E6FF5B
:104300003AC1E6FF3BC1E6FF1EEF1DF03D0E4E6ECB
:104310008B0E59EC1CF03CC1E6FF3DC1E6FF3EC1EF
:10432000E6FF3FC1E6FF1EEF1DF059EC1CF0E5C1B2
:10433000E6FFE6C1E6FFE7C1E6FFE8C1E6FF7BDE98
:1043400056EF1DF04FC0E6FF50C0E6FF51C0E6FF3C
:104350001200E90EE66E010E58DE2BEF22F055DE5C
:10436000E90EE66E010EFEEF1FF04EC0DFFF010EFC
:104370004FC0DBFF020E50C0DBFF030E51C0DBFF5E
:104380001200E66E060E53EC1CF0010E1200E55210
:10439000E552E55212004EC041F04FC042F050C00D
:1043A00043F051C044F01200010EDBCF4EF04F6AD3
:1043B00050DE19EF21F0C9C140F0CAC141F0CBC1B4
:1043C00042F0CCC143F0120043D823EF1EF080DD51
:1043D000010F6FEF20F0D9CFE9FFDACFEAFF12002B
:1043E0002F0D05014BEF20F0560E4E6E8B0E59EC43
:1043F0001CF099EF1EF0420E4E6E8B0E59EC1CF025
:10440000A2EF1EF02CDED950120041DE61DDC0EFBC
:1044100020F014D81E0E59EF1DF010D8160E59EFCB
:104420001DF0EE52260E59EF1DF0E126DF6A010E57
:10443000DB6A1200E66E070E53EF1CF075EC1CF001
:10444000EE521200E66AD10EE66E010E05EF20F084
:10445000E66A11EF1DF0ED0EE66E010ECFDDD7EF2F
:0C4460001FF0D90EE66E010E05EF20F0F3
:04446C00D8CFE4FFC2
:10447000E0CFE4FFE46EDACFE4FFE9CFE4FFEACF78
:10448000E4FFF3CFE4FFF4CFE4FFE65239EC37F07A
:10449000A4A645D1A4960001602B00019B51000108
:1044A000605D01E29FD0606B000151EC36F0EF6A75
:1044B00079907B6A7A6A0001992B00019A51000178
:1044C000995D01E3996BD5EC37F0EA22EE50ED10DF
:1044D00001E188D0BEEC37F0EECF58F0EFCF59F0C5
:1044E0005850561802E1595057185FE009B28986B2
:1044F0000DEC37F0EA22EE50ED1051E0BEEC37F053
:104500000401EE50565CCF6FEE505758D06FE83430
:1045100022E2CF510008000ED0551DE200010DEC43
:1045200037F0D0EC35F004015750D019E8AE02D086
:10453000D03504D0CF51565CD05157580AE2000113
:104540000DEC37F0E9EC36F05650EE265750ED22E0
:104550002CD0000124D0CFC456F0D0C457F0566CF4
:10456000571E000E572200010DEC37F0EA22EECF65
:1045700058F0EFCF59F059505718E8AE02D05734E1
:1045800004D05650585C5750595809E20DEC37F09A
:10459000E9EC36F05650EE5E5750ED5A06D0BEECC0
:1045A00037F056C0EEFF57C0EDFF51EC36F0120E5B
:1045B000EF6EF29E00015EEC37F057C056F0576A7E
:1045C0005650B66E5EEC37F05650B56EF00EB41421
:1045D0000009B46EF00EB4140909B46E7980F28E3D
:1045E00009B289960401000ED8807A55000E7B55D9
:1045F0002EE2882B000E89237A51885D7B518959E0
:1046000026E3886B896B030E7E5D1FE27C51EA6AAC
:10461000200FE96E010EEA2280CFEFFF7C51EA6A9B
:10462000230FE96E010EEA2281CFEFFF7C51EA6A87
:10463000260FE96E010EEA2282CFEFFF7C2B030EDC
:104640007C5D01E37C6B7E2B02D07A6B7B6B000E72
:10465000D8807F55000E80551CE2000ED8808E5504
:10466000000E8F5516E28A2B000E8B237F518A5D38
:1046700080518B590EE38A6B8B6B030E835D07E2CF
:10468000812B030E815D01E3816B832B02D07F6B55
:10469000806B8E518F110BE0050E8D5D07E3C18C91
:1046A0009E9C9D8CC280C2828D6B01D08D2B01019E
:1046B000BE5101E0BE070401BE51BF11C011C111BE
:1046C0000BE0BE07000EBF5BC05BC15BBE51BF11FC
:1046D000C011C11101E18996020E955D20E198514A
:1046E00099111DE09807000E995B9851991117E1F7
:1046F0009A519B1114E09A07000E9B5B9A519B11F3
:104700000AE1045003E18D808B8202D08C82898281
:10471000030E956F04D0E80E986F030E996F9EAC50
:104720004FD09E9CC1AC07D0C19C010E0401906F7C
:10473000916B8C6B2AD0C450586E596E586AC35016
:1047400000015810566E59C057F004018C51E96EA3
:10475000EA6A22EC37F0EA2256C0EEFF57C0EDFFBE
:104760000B0E8C5D0EE18C51E96EEA6A22EC37F09B
:10477000D0EC35F09251565C9351575802E2010E3D
:10478000946FD890903791378C2B100E8C5D0EE281
:1047900090518E15566E91518F15576E5650571079
:1047A00005E18C2BD89090379137EFD7100E8C5DA8
:1047B00002E39D9C05D08C51040DF328C26EC28289
:1047C000E552E552E7CFD9FFE552E5CFF4FFE5CF5B
:1047D000F3FFE5CFEAFFE5CFE9FFE5CFDAFFE550EC
:1047E000E5CFE0FFE5CFD8FF1000D9CFE6FFE1CF5E
:1047F000D9FF020EE126DE6ADD6AE2CFD1F4E1CF15
:10480000D2F4D1C44EF04EC04FF04E6A0401D251E2
:1048100004014E10D36F4FC0D4F4D3C4DEFFD4C410
:10482000DDFF080EDE26000EDD22D9CFE9FFDACF4C
:10483000EAFFBF0ED880EE540E0EED540BE3DECF30
:10484000E9FFDDCFEAFFEE0EEF6EDF2A010E01E396
:10485000DB2AEBD7020EE15C02E2E16AE552E16E8F
:10486000E552E7CFD9FF1200DEEC37F0BF0EF36E52
:10487000010EF3CFDBFF0E0EF36E020EF3CFDBFF64
:10488000F28C010EDBCFE9FF020EDBCFEAFFEF5027
:10489000EE0806E1010EDB06020EF3E2DB06F1D7BD
:1048A000AEEC36F004014E50CD5D4F50CE5906E2CD
:1048B000010EDBCFCDF4020EDBCFCEF4F28C030E73
:1048C000E15C02E2E16AE552E16EA7EF35F0ECEC63
:1048D00037F0896A926804018E6B8F6B8A6A9368DD
:1048E0008B6A94688C968C9495969594928E010E12
:1048F000BD6F846B826B816B836B7D6B7C6B7E6B1E
:104900007A6B7B6B7F6B806B886B896B8A6B8B6B35
:104910008C6B76827680769C769A76887696FA0E7E
:10492000776EDE6ADD6A64EC36F0100E4E5C000EC7
:104930004F5813E269EC36F0010ED890E936EA36AA
:10494000E806FBE1000EE926010EEA22EE6AED6AB6
:10495000DF2A010EE8E3DB2AE6D70401B76BB86B68
:10496000B56BB66BDE6ADD6A79EC37F00AE269ECAA
:1049700036F0000EE926020ED8EC36F0F5E3DB2A1D
:10498000F3D7DE6ADD6A79EC37F00AE269EC36F0DB
:10499000400EE926020ED8EC36F0F5E3DB2AF3D719
:1049A000DE6ADD6A64EC36F0000E4E5C010E4F5894
:1049B0000AE269EC36F0000EE926030ED8EC36F078
:1049C000F1E3DB2AEFD70401B96BBA6BBB6BBC6BAD
:1049D000856B866B876B0F01498FBE0EC16ED08EC3
:1049E0007694A386A596B9EC0CF0B7EC3EF07684ED
:1049F0003EEC32F00401C96BCA6BCB6BCC6B0E6A18
:104A0000BE6BBF6BC06BC16B600EC26FEA0EC36F33
:104A1000C46BC56B010EC66FCD6BCE6B926B936B87
:104A2000966B976B986B996B9A6B9B6B956B946B72
:104A3000F28EF28C020EE15C02E2E16AE552E16E76
:104A4000A7EF35F0A2EC35F0050EE126B5EC36F017
:104A5000BAEC34F004017E5100080AE2CCEC2EF0EE
:104A600004017D2B030E7D5D01E17D6B7E07F2D796
:104A7000835100080AE2E9EC2EF00401822B030EB8
:104A8000825D01E1826B8307F3D7200E0501E76E9B
:104A9000BC19E8AE02D0E73402D0E750BC5D01E2B9
:104AA0002AD16550020B01E026D1400EE66E400E81
:104AB000E66E020EE66EADEC43F0E2EC37F0E76E28
:104AC000020EE7CFDBFFDB50000801E3B8D0030E96
:104AD000DB6A020EDB50F36E030E6EEC36F001E380
:104AE000AED09EEC36F0040EEFCFDBFF0401EC51AC
:104AF00014E056EC37F0040EDBCFEFFFB72B030EBC
:104B0000DB2A0401EC07EC5137E109B08B80ADECF6
:104B100019F009A02FD08B902DD0EB512DE0040E71
:104B2000DB50590829E1EB6B1C0EEC6F020EDBCF5A
:104B3000E6FF030EDB50E552E75C4E6E1C0E4E5C4A
:104B40001BE3030EDB2AEC510FE09EEC36F0EF5036
:104B5000E66E56EC37F0E552E750EF6EB72B030EDA
:104B6000DB2A0401EC07EFD709B08B80ADEC19F01C
:104B700009B08B90BCEC36F009A806D0040EDBCF50
:104B8000E6FF13EC4CF0E5520401EC5155E1E7511E
:104B90001BE10D0E4E6E040EDB504E5C06E00A0E5D
:104BA0004F6E040EDB504F5C0FE1010EE76F56ECC9
:104BB00037F00D0EEF6EB72B09B08B80F9D809B026
:104BC0008B90BCEC36F02BD0040EDB5008080FE1C4
:104BD0000401B75100080BE2B707B75191EC35F06B
:104BE000EF6A010E4E6E8D0E84EC35F018D0040E77
:104BF000DB500D0814E0040EDB500A0810E0200E14
:104C0000F36E040E6EEC36F00AE356EC37F0040E49
:104C1000DBCFEFFF0401E76BEB6B0401B72B040163
:104C2000B7514E6E4F6A000E4E1806E1010E4F1836
:104C300003E18487B76BB86B030EDB2A4AD7040104
:104C4000845139E084A105D0FD0E4E6E8C0E0AEC25
:104C500037F0040184A305D0E00E4E6E8C0E0AECF2
:104C600037F0040184A505D0C60E4E6E8C0E0AECFA
:104C700037F0040184A705D0AC0E4E6E8C0E0AEC02
:104C800037F0040184A905D08F0E4E6E8C0E0AEC0D
:104C900037F0040184AD05D06F0E4E6E8C0E0AEC19
:104CA00037F0040184AF05D0570E4E6E8C0E0AEC1F
:104CB00037F00401846BCA511DE0010E0E1414E09C
:104CC000CB5112E1380E4E6E8C0E84EC35F0020E94
:104CD000E66EC9C44EF04F6AABEC35F08EEC35F0A1
:104CE0000401010ECB6F06D0010E0E1403E1CB516F
:104CF00001E0CB6B37D8050EE15C02E2E16AE552D8
:104D0000E16EA7EF35F039EC37F0B5C4DFFFDF2AED
:104D1000400EDFEC35F001E1DF6A0401B651DF5CE3
:104D200001E120D80401B551EA6A000FE96E020ED4
:104D3000EA22FE0EDBCFEFFFB52B400EB55D01E1A1
:104D4000B56BB651B55D01E18485FE0EDBCF4EF04B
:104D50004F6A4EBE4F684EC0F3FF4FC0F4FFE5529E
:104D6000A7EF35F039EC37F00401B551B65D1DE021
:104D70000501A45105E039EC44F07EEC38F0F8D799
:104D80000401B651D880B55507E2B651B55D12ECB5
:104D900036F0B5C4B6F407D0400ED880B65512EC44
:104DA00036F00401B66B39EC44F0E552A7EF35F06C
:104DB000A2EC35F0090EE126DE6ADD6A020EDB6A3E
:104DC000030EDB6A050EDB6A010EF36E060EF3CFEF
:104DD000DBFF0401C76BC86BCC5101E18CD0060E20
:104DE000DB6A040EB7C4DBFFDB5003E0040EDB0616
:104DF00002D0040EDB687FEC37F016E0050EF36E90
:104E0000DBCFF4FFE850F45C0FE2040EDB50B85D3A
:104E10000BE0040EDB5003E0040EDB0602D0040EB0
:104E2000DB68050EDB2AE7D77FEC37F05BE1070E86
:104E3000B8C4DBFF040EDBCFB8F4E66AD950020F2A
:104E4000E2EC36F0070EDBCFB8F4080EB8C4DBFF97
:104E5000040EDB50F36E080EDB50F35C19E0080E15
:104E6000DB5091EC35F0030EDBCFE7FFEF50E72688
:104E7000030EE7CFDBFF080EDB2ADB504E6E4F6AD6
:104E8000E850E6E1010E4F18E3E1080EDB6AE0D7D7
:104E9000030EDB1C010FE76E030EE7CFDBFF020EF4
:104EA000DB50F36E030EDB50F35C0CE1010EF36E8E
:104EB000060EF3CFDBFF040EDB5091EC35F00D0E48
:104EC000EF6E19D0120E4E6E8C0E84EC35F0030E80
:104ED00084EC36F04EC0E6FFEDEC36F0D9EC46F04F
:104EE000E55205D0E90E4E6E8B0E29EC37F0E2EC60
:104EF00037F08EEC35F0060EDB5001E168D204018C
:104F000000EC38F0A6EC36F0F3CFC7F40401B4ECB3
:104F100035F004E1010E4F1801E1B86BC751DE6EA8
:104F2000DD6AE6EC36F02C0823E0E6EC36F00D08FE
:104F30001FE0E6EC36F00A081BE000EC38F0A6ECC7
:104F400036F0F3CFC8F40401B4EC35F004E1010EFF
:104F50004F1801E1B86BC7C451F0506AC851000145
:104F600050244E6E000E51204F6E4EC0DEFFDD6E9F
:104F7000000EDFCF42F0010EDBCF43F0520E42189D
:104F800002E1540E431801E1F1D1550E421802E13D
:104F9000510E431801E1E8D14D0E421802E1480ECE
:104FA000431801E1DED1520E421802E1530E4318BC
:104FB00001E1D4D1520E421802E1510E431801E131
:104FC000CAD1420E421802E1520E431801E1C0D18B
:104FD000540E421802E1510E431801E1B6D1540EAD
:104FE000421802E1530E431801E1ACD1530E4218AE
:104FF00002E1430E431801E1A2D1530E421802E12F
:10500000510E431801E198D14D0E421802E1580E9D
:10501000431801E18ED1530E421802E1450E4318A8
:1050200001E184D1430E421802E1410E431801E12F
:105030007AD14D0E421802E1510E431801E170D1B0
:10504000320E421802E1530E431801E166D1450EBB
:10505000421802E1530E431801E15CD1470E421899
:1050600002E1510E431801E152D1430E421802E110
:10507000510E431801E148D14B0E421802E1430E94
:10508000431801E13ED14C0E421802E1420E431892
:1050900001E134D1440E421802E14E0E431801E101
:1050A0002AD1490E421802E14E0E431801E120D1E7
:1050B000420E421802E1510E431801E116D14C0E86
:1050C000421802E1510E431801E10CD14C0E421876
:1050D00002E1530E431801E102D14E0E421802E1E3
:1050E000510E431801E1F8D04E0E421802E1530E62
:1050F000431801E1EED0430E421802E1530E43186B
:1051000001E1E4D04D0E421802E1450E431801E1E1
:10511000DAD0450E421802E1510E431801E1D0D019
:10512000500E421802E1510E431801E1C6D0500E54
:10513000421802E1540E431801E1BCD0500E42184F
:1051400002E1530E431801E1B2D04D0E421802E1C4
:10515000530E431801E1A8D0570E421802E14D0E3C
:10516000431801E19ED0520E421802E14D0E431841
:1051700001E194D0440E421802E1500E431801E1BF
:105180008AD04F0E421802E1500E431801E180D040
:10519000490E421802E1500E431801E176D0410E4B
:1051A000421801E143506EE0560E421801E14350AF
:1051B00066E0490E421801E143505EE04F0E42188E
:1051C00001E1435056E0550E421802E1430E4318E8
:1051D0004EE0430E421801E1435046E0520E4218A1
:1051E00001E143503FE04D0E421802E14C0E4318DE
:1051F00036E0330E421802E1540E43182DE0440EFF
:10520000421802E1540E431824E0330E421802E122
:105210004C0E43181BE0540E421802E14C0E43188A
:1052200012E04D0E421802E1430E431809E004015A
:10523000C85101E09ED061EC37F067EC37F0ADD09B
:10524000B8EC11F0B2D04FEC0FF0AFD082EC0EF012
:10525000ACD0BEEC0EF0A9D039EC0FF0A6D049ECE2
:105260000EF0A3D0FFD8A1D0E6EC2DF09ED001D94E
:105270009CD096EC2EF099D0CCEC2EF096D0E2ECAF
:105280002EF093D0E9EC2EF090D025EC30F08DD0BC
:105290009AEC30F08AD089EC2FF087D06AEC2FF0AE
:1052A00084D04FEC2FF081D0A4EC11F07ED042ECF2
:1052B00016F07BD01CEC16F078D09CEC15F075D075
:1052C000B4EC15F072D0F9EC16F06FD088EC0DF05C
:1052D0006CD059EC17F069D07AEC17F066D08CECF2
:1052E00017F063D0ACEC17F060D0D3EC17F05DD0C2
:1052F00037EC17F05AD04AEC17F057D04EEC31F09B
:1053000054D0A0EC31F051D0E7EC17F04ED000ECC7
:1053100018F04BD033EC18F048D02CEC3FF045D0CF
:105320002BEC19F042D07CEC2EF03FD04DEC15F078
:105330003CD01BEC14F039D06CEC19F036D0A8EC52
:1053400019F033D081EC32F030D0B5EC32F02DD002
:1053500056EC31F02AD05DEC31F027D06DEC31F015
:1053600024D0D3EC12F021D0AEDB1FD040EC13F0F0
:105370001CD061EC37F0C8C4E6FFC5DCE55267EC31
:1053800037F075EC37F0C7C4E6FFEDEC36F085EC8E
:1053900037F0020EE66EC8C44EF04F6AABEC35F043
:1053A000270EC7EC35F08EEC35F00401E6EC36F054
:1053B0000D080DE084510BE1520E4E6E4F6ADF5026
:1053C0004E1803E1DE52DD504F1801E0848FB7C460
:1053D000B8F4090EE15C02E2E16AE552E16EA7EF82
:1053E00035F039EC37F02C0EDF6E010E0101C315DC
:1053F00003E1FE0EDB5010E08DEC36F00401C851E5
:1054000004E0C8C4E6FF7FDCE552FD0EDB5004E09B
:10541000DFCFE6FF78DCE552E552A7EF35F0A2ECEE
:1054200035F00101C3A104D0CD0E4E6E8B0E16D007
:105430000401BD5108E0FE0EDB5005E1CA0E4E6EC0
:105440008B0E84EC35F0FE0EDB50020804E1C70E33
:105450004E6E8B0E03D0C40E4E6E8B0E84EC35F068
:10546000A7EF35F0F0EC37F0D6EC35F07BDC67EFEA
:1054700024F0D9CFE6FFE1CFD9FF040EE126E66A9A
:10548000E66AAFDFE552E552E66AD9CFE6FFDACF4A
:10549000E6FF030EE66E11EC33F0E552E552E552FD
:1054A000E552E66AD950020FE66E000EDA20E66E8B
:1054B000020EE66E11EC33F0E552E552E552E5528C
:1054C0000401845101E0F5D2010E4E6E4F6ADF50A7
:1054D0004E1803E1DE52DD504F181AE1D950020F89
:1054E000E96EDACFEAFFEE50ED100BE0010E4E6EE2
:1054F0004F6A020EDB504E1803E1030EDB504F18CB
:1055000004E1020EDBCFBDF402D00401848DCED2C3
:10551000020E4E6E4F6ADF504E1803E1DE52DD5030
:105520004F181AE1D950020FE96EDACFEAFFEE50B8
:10553000ED100BE0010E4E6E4F6A020EDB504E185E
:1055400003E1030EDB504F1804E1020EDBCFC2F182
:1055500002D00401848DAAD2030E4E6E4F6ADF5032
:105560004E1803E1DE52DD504F181CE1D950020FF6
:10557000E96EDACFEAFFEE50ED1003E106908C946D
:1055800010D0010E4E6E4F6A020EDB504E1803E132
:10559000030EDB504F1803E106808C9402D0040107
:1055A000848D84D2040E4E6E4F6ADF504E1803E194
:1055B000DE52DD504F181DE1020EDBCF4EF0030E20
:1055C000DBCF4FF04F3404E24E502008000E4F5412
:1055D00007E2200EF36E020EF3CFDBFF030EDB6A51
:1055E000E3EC18F0000901E0FBD7020EDB50136E6C
:1055F0005DD20A0E4E6E4F6ADF504E1803E1DE5246
:10560000DD504F181CE1D950020FE96EDACFEAFFE6
:10561000EE50ED1003E10101C39110D0010E4E6E6A
:105620004F6A020EDB504E1803E1030EDB504F1899
:1056300003E10101C38102D00401848D37D2320E0F
:105640004E6E4F6ADF504E1803E1DE52DD504F18A8
:105650000FE1D950020FE96EDACFEAFFEE50ED10FC
:1056600003E10401C66B03D00401010EC66F1ED214
:10567000330E4E6E4F6ADF504E1803E1DE52DD509E
:105680004F1811E1FF0EE76E020EDBCF4EF0030E56
:10569000DBCF4FF0E7504E164F6A4E500C6E0C5059
:1056A00001E10E9003D2340E4E6E4F6ADF504E1859
:1056B00003E1DE52DD504F180EE1FF0EE76E020EE1
:1056C000DBCF4EF0030EDBCF4FF0E7504E164F6AA4
:1056D0004E500D6EEBD1350E4E6E4F6ADF504E18A8
:1056E00003E1DE52DD504F1814E1010E4E6E4F6A99
:1056F000020EDB504E1803E1030EDB504F1804E19D
:105700000401010ECA6F04D00401CA6B0401CB6B03
:10571000CDD1360E4E6E4F6ADF504E1803E1DE5289
:10572000DD504F1812E1010E4E6E4F6A020EDB5033
:105730004E1803E1030EDB504F1804E10401010E83
:10574000CC6F02D00401CC6BB1D13C0E4E6E4F6ACF
:10575000DF504E1803E1DE52DD504F180DE1020E0E
:10576000DBCF92F4030EDBCF93F4FF0E040192170C
:10577000030E040193179AD13D0E4E6E4F6ADF500F
:105780004E1803E1DE52DD504F1837E1F29EF29CD5
:10579000020EDBCF96F4030EDBCF97F40401965193
:1057A000971109E10401956B0401986B996B040151
:1057B0009A6B9B6B1FD004019551030A14E0020AF7
:1057C0000FE0010A0DE0020A01E00AD096C49AF443
:1057D00097C49BF40401E80E986F030E996F0AD0EA
:1057E0000401010E956F0401986B996B04019A6B8B
:1057F0009B6B00D0F28CF28E59D1FA0E4E6E4F6A2E
:10580000DF504E1803E1DE52DD504F181EE1D95033
:10581000020FE96EDACFEAFFEE50ED1002E10992D5
:1058200013D0010E4E6E4F6A020EDB504E1803E18C
:10583000030EDB504F1806E10982959295909292E3
:10584000929602D00401848D31D1FB0E4E6E4F6AC8
:10585000DF504E1803E1DE52DD504F182BE1D950D6
:10586000020FE96EDACFEAFFEE50ED1003E1099680
:1058700009941FD0010E4E6E4F6A020EDB504E1877
:1058800003E1030EDB504F1812E109840996EC0E78
:10589000E66E3EEC4CF0E552020EE66EE66A1C0E39
:1058A000E66E38EC4BF0E552E552E55202D00401C9
:1058B000848DFCD0FC0E4E6E4F6ADF504E1803E113
:1058C000DE52DD504F182BE1D950020FE96EDACFCE
:1058D000EAFFEE50ED1003E1099609941FD0010E86
:1058E0004E6E4F6A020EDB504E1803E1030EDB5082
:1058F0004F1812E109860984EC0EE66E3EEC4CF07E
:10590000E552020EE66EE66A1C0EE66E38EC4BF0CF
:10591000E552E552E55202D00401848DC7D0FD0E58
:105920004E6E4F6ADF504E1803E1DE52DD504F18C5
:1059300029E1D950020FE96EDACFEAFFEE50ED10FF
:1059400002E109981ED0010E4E6E4F6A020EDB5026
:105950004E1803E1030EDB504F1811E10988EC0EDD
:10596000E66E3EEC4CF0E552020EE66EE66A1C0E68
:10597000E66E38EC4BF0E552E552E55202D00401F8
:10598000848D94D0FE0E4E6E4F6ADF504E1803E1A8
:10599000DE52DD504F181AE109829592959092924D
:1059A0008C908C808C908C808C908C808C908C8057
:1059B0008C908C808C908C808C908C808C908C8047
:1059C0008C908C808C908C80EBD770D04E684F6A16
:1059D000DF504E1803E1DE52DD504F181AE1D95066
:1059E000020FE96EDACFEAFFEE50ED1002E1099AFC
:1059F0000FD0010E4E6E4F6A020EDB504E1803E1BF
:105A0000030EDB504F1802E1098A02D00401848D95
:105A10004DD04E6A010E4F6EDF504E1803E1DE523C
:105A2000DD504F181AE1D950020FE96EDACFEAFFC4
:105A3000EE50ED1002E1099C0FD0010E4E6E4F6A40
:105A4000020EDB504E1803E1030EDB504F1802E14B
:105A5000098C02D00401848D29D0010E4E6E010EF6
:105A60004F6EDF504E1803E1DE52DD504F181CE13F
:105A7000D950020FE96EDACFEAFFEE50ED1003E1E4
:105A80000990948010D0010E4E6E4F6A020EDB50CA
:105A90004E1803E1030EDB504F1803E10980949088
:105AA00002D00401848D02D00401848DE66AB7DC43
:105AB000E552040EE15C02E2E16AE552E16EE55274
:105AC000E7CFD9FF120039EC37F04CEC37F0010E7C
:105AD00087EC35F00401845176E1DF0406E1020E23
:105AE000E66EC9C44EF04F6A18D0020EDFEC35F0F6
:105AF00006E1200EE66EE66AE66AE66A3ED0030E2E
:105B0000DFEC35F002E1135020D0040EDFEC35F06D
:105B100007E134EC24F0C3EC36F0ABEC35F04DD0BB
:105B2000050EDFEC35F00CE1C3EC36F0ABEC35F0F4
:105B30008EEC35F0F29C0401CD6BCE6BF28C41D033
:105B4000060EDFEC35F004E10F5008EC36F013D010
:105B50003C0EDFEC35F005E192C44EF093C44FF0FB
:105B600008D03D0EDFEC35F00BE196C44EF097C443
:105B70004FF0F4EC37F0EDEC36F0D1EC37F01DD00F
:105B8000C80EDFEC35F01CE1F29E1EC0E6FF1FC020
:105B9000E6FF20C0E6FF21C0E6FFD1EC37F02C0E77
:105BA000C7EC35F022C0E6FF23C0E6FF24C0E6FFC5
:105BB00025C0E6FFD1EC37F0F28E8EEC35F001D047
:105BC000848DD6EC35F0E552A7EF35F0A2EC35F038
:105BD000050EF4EC36F0010EB3EC37F0B7EC37F00D
:105BE000E66AD950030FE2EC36F0E66AD950040FAA
:105BF0000AEC38F010E1DF50926E010EDB50936E2C
:105C0000020EDB50946E030EDB50956E040EDB50DB
:105C1000966ED6EC35F0050EE15C02E2E16AE552E3
:105C2000E16EA7EF35F0A2EC35F0FE0EDB50100868
:105C300005E2100EF36EFE0EF3CFDBFFFD0EDB5020
:105C40002BE0FE0EDB505DEC4CF0F35004018E13A4
:105C5000F4508F13080EF36EFE0E6EEC36F00DE26C
:105C6000010EF36EFE0EDB5003E0CCEC35F0FDE1EF
:105C7000F350F31C0F0148173DD0FE0EDB500C080B
:105C800039E3CAEC36F004E0E846FE0B4E06FCE1D0
:105C9000E81C0F0149172ED0FE0EDB505DEC4CF0D6
:105CA000F3CF4EF0F4CF4FF04E1E4F1E4E50040176
:105CB0008E174F508F17080EF36EFE0E6EEC36F0F7
:105CC0000CE2010EF36EFE0EDB5003E0CCEC35F07F
:105CD000FDE1F3500F0148130DD0FE0EDB500C0810
:105CE00009E3CAEC36F004E0E846FE0B4E06FCE1A0
:105CF0000F014913A7EF35F00EEC38F0B3EC37F095
:105D0000010F0AEC38F00AE1010EDBCFE6FFDFCF2E
:105D1000E6FF89DFE552E552D6EC35F0020EE15C94
:105D200002E2E16AE552E16EA7EF35F00EEC38F0E1
:105D300087EC35F023EC36F027E1010EDB5002E171
:105D4000DF50896E01EC37F01FE1010EDB5002E1FC
:105D5000DF508A6E01EC37F017E1010EDB5002E1F3
:105D6000DF508B6E01EC37F00FE1010EDB5002E1EA
:105D7000DF508C6E01EC37F007E1010EDB5002E1E1
:105D8000DF508D6ED6EC35F0020EE15C02E2E16A86
:105D9000E552E16EA7EF35F0010EE66EE66E12EC0D
:105DA00037F0805006EC37F0815006EC37F0825027
:105DB00006EC37F0835006EC37F08450F9EC37F0FE
:105DC0008EEF35F05FEC36F0980E4E6E940E0AEFC3
:105DD00037F0DEEC37F0DF6A010EF36EDB6E020E99
:105DE000DB6AE66A010EE66E12EC37F09DBCFED768
:105DF000DF6ADFCF4EF0100EE76E4E18E8AE02D02D
:105E0000E73402D0E7504E5C3FE2010EDB50040164
:105E10008E1500014E6E020EDB5004018F1500013D
:105E20004F6E4E504F1023E02C0EC7EC35F0DFCFF5
:105E30004EF075EC37F04EAE03D04F6850685168A5
:105E40004EC0E6FF8BEC35F03A0EC7EC35F0DFCFF5
:105E5000E9FFEA6AE9BEEA6822EC37F0EA22EECF0F
:105E60004EF0EFCF4FF0F4EC37F08BEC35F0AEECBA
:105E700036F0D8904E364F36010E4EC0DBFF020E84
:105E80004FC0DBFFDF2AB5D7020EA4EC37F0030EBC
:105E9000E15C02E2E16AE552E16EA7EF35F0DAEC8F
:105EA00037F0030EB3EC37F0020F0AEC38F00AE1DA
:105EB0008CEC37F005E269EC36F0020EDBCFEFFF39
:105EC000D6EC35F0030EE15C02E2E16AE552E16EE8
:105ED000A7EF35F0DEEC37F04CEC37F0030E87EC33
:105EE00035F0040184510DE18CEC37F005E269ECEA
:105EF00036F0020EEFCFDBFF020E84EC36F0FCEC46
:105F000036F0030EE15C02E2E16AE552E16EA7EFD2
:105F100035F003EC38F001E090D0020EDB500108C0
:105F200001E287D0010EDB50070801E282D0410E6A
:105F3000DFEC35F016E1020EDB500AE1DBEC35F068
:105F400003E0CCEC35F0FDE1F350F31C921673D076
:105F5000DBEC35F003E0CCEC35F0FDE1F3509212D0
:105F60006AD0420EDFEC35F016E1020EDB500AE19A
:105F7000DBEC35F003E0CCEC35F0FDE1F350F31C45
:105F8000931659D0DBEC35F003E0CCEC35F0FDE1B5
:105F9000F350931250D0430EDFEC35F016E1020EB1
:105FA000DB500AE1DBEC35F003E0CCEC35F0FDE151
:105FB000F350F31C94163FD0DBEC35F003E0CCEC4F
:105FC00035F0FDE1F350941236D0440EDFEC35F09D
:105FD00016E1020EDB500AE1DBEC35F003E0CCEC1D
:105FE00035F0FDE1F350F31C951625D0DBEC35F0D0
:105FF00003E0CCEC35F0FDE1F35095121CD0450EDA
:10600000DFEC35F016E1020EDB500AE1DBEC35F097
:1060100003E0CCEC35F0FDE1F350F31C96160BD009
:10602000DBEC35F003E0CCEC35F0FDE1F3509612FB
:1060300002D0848D02D0D6EC35F0030EE15C02E292
:10604000E16AE552E16EA7EF35F0DEEC37F0020EC3
:10605000DB6A4CEC37F0050EB3EC37F0010F0AECBD
:1060600038F060E1010EDB50070850E3410EDFEC31
:1060700035F00AE1DBEC35F003E0CCEC35F0FDE186
:10608000F350801439E029D0420EDFEC35F00AE1FC
:10609000DBEC35F003E0CCEC35F0FDE1F35081149E
:1060A0001CE12AD0430EDFEC35F00AE1DBEC35F0E1
:1060B00003E0CCEC35F0FDE1F35082140EE11CD08E
:1060C000440EDFEC35F00BE1DBEC35F003E0CCEC1B
:1060D00035F0FDE1F35083140FE0010E10D0450EB2
:1060E000DFEC35F013E1DBEC35F003E0CCEC35F020
:1060F000FDE1F350841402E1000E01D0010EE76EC1
:10610000020EE7CFDBFFDB5008E002D0848D0AD01F
:10611000010EF36E020EF3CFDBFF020E84EC36F0BD
:10612000FCEC36F0030EE15C02E2E16AE552E16E5E
:10613000A7EF35F003EC38F001E090D0020EDB5011
:10614000010801E287D0010EDB50070801E282D08E
:10615000410EDFEC35F016E1020EDB500AE1DBEC1C
:1061600035F003E0CCEC35F0FDE1F350F31C89167B
:1061700073D0DBEC35F003E0CCEC35F0FDE1F3500F
:1061800089126AD0420EDFEC35F016E1020EDB50C8
:106190000AE1DBEC35F003E0CCEC35F0FDE1F35047
:1061A000F31C8A1659D0DBEC35F003E0CCEC35F06B
:1061B000FDE1F3508A1250D0430EDFEC35F016E1CA
:1061C000020EDB500AE1DBEC35F003E0CCEC35F0FD
:1061D000FDE1F350F31C8B163FD0DBEC35F003E010
:1061E000CCEC35F0FDE1F3508B1236D0440EDFECF1
:1061F00035F016E1020EDB500AE1DBEC35F003E08E
:10620000CCEC35F0FDE1F350F31C8C1625D0DBEC23
:1062100035F003E0CCEC35F0FDE1F3508C121CD0EE
:10622000450EDFEC35F016E1020EDB500AE1DBEC47
:1062300035F003E0CCEC35F0FDE1F350F31C8D16A6
:106240000BD0DBEC35F003E0CCEC35F0FDE1F350A6
:106250008D1202D0848D02D0D6EC35F0030EE15CB5
:1062600002E2E16AE552E16EA7EF35F0D9CFE6FF31
:10627000E1CFD9FFE652DF6AFF0EDF5C0AE2E86891
:10628000E85005E0E80600D000D000D0F9D7DF2ABA
:10629000F3D7E552E552E7CFD9FF1200F29EF29C08
:1062A0006592656AE3DF0FEF00F01200F29EF29C48
:1062B0006592656ADBDFFF0012005FEC36F080500C
:1062C000080B01E0010EF9EC37F00101C3B103D076
:1062D000020EA4EC37F0D6EF35F0A2EC35F0060E46
:1062E000F4EC36F0070E87EC35F0010EE66ED9506F
:1062F000040FE2EC36F0E76E050EE7CFDBFF04019A
:10630000845116E1DFCFC2F4010EDBCFC3F4020EDD
:10631000DBCFC4F4030EDBCFC5F4050EDB5006E182
:10632000040EDB5002E0898601D08996D6EC35F068
:10633000060EE15C02E2E16AE552E16EA7EF35F09C
:10634000A2EC35F0100EE126F0EC37F0E7DBE66A60
:10635000D950010FAFEC35F0E66A63D9F9EC36F0AD
:10636000E66AA9EC37F0010EB3EC37F0040FAFEC9E
:1063700035F0020EB3EC37F0020FF1DB030EB3EC95
:1063800037F00A0FECDB060EB3EC37F0060FE7DB55
:10639000070EB3EC37F00E0FE2DB040EB3EC37F070
:1063A0000F0FDDDB050EB3DBBC0E4E6E8B0EACDBD0
:1063B000010E84EC36F04EAE03D04F685068516841
:1063C000C4EC37F0B40E4E6E8B0E9EDBDFCF4EF07A
:1063D00075EC37F0FCEC36F0AC0E4E6E8B0E94DBA9
:1063E000040EDBCF4EF0050EDBCF4FF0506A516A42
:1063F0004FAE02D050685168C4EC37F0A40E4E6E18
:106400008B0E82DB020EDBCF4EF0030EDBCF4FF0A4
:10641000506A516AFCEC36F09C0E4E6E8B0E74DBAB
:10642000D9500A0FA8DB13EC38F051EC37F0D950F3
:10643000060FA1DBD1EC37F071DB8C0E4E6E8B0EAC
:1064400063DB0E0E6EEC37F0840E4E6E8B0E5CDB53
:106450000F0E6EEC37F051EC37F0080EE66E17ECCD
:1064600037F051EC37F0E66A17EC37F09FDB100E8F
:10647000E15C02E2E16AE552E16E69D339EC37F0A2
:10648000DF6A110EDF5C04E2B3DBEF6ADF2AF9D7C3
:1064900092EC37F0DF6A100EDF5C21E2A9DBEF50EF
:1064A00080081DE3A5DBEFCF4EF0200E4E5C17E316
:1064B0009FDBEF50E66E180E02014F6AFA254E6E12
:1064C000FB5178EC36F094DBEF50E66E020E4F6A2B
:1064D000FC254E6EFD5178EC36F0DF2ADCD7DF501C
:1064E000E824180FFAC2E9FFFBC2EAFFEF6EDF50A3
:1064F000E824020FFCC2E9FFFDC2EAFFEF6EE5529D
:1065000026D3ECEC37F0DF6AF0EC37F0010EDB6AF3
:10651000110EF36E010EE2DB0BE2010EDB50EA6AB4
:10652000D50FE96E040EEA22EF6A010EDB2AF0D7DE
:10653000100EE66EAEEC37F038D8E2EC37F0DF6ED6
:10654000E668FB0EE66EE66A97EC37F0D0EC49F0B1
:10655000F0DB49DB9AEC47F0ECDB28DB020EE15C78
:1065600002E2E16AE552E16EF2D239EC37F0A7DBE4
:10657000DF6A110EDF5C04E23BDBEF6ADF2AF9D74A
:1065800092EC37F0800E0401D55D09E2D551200868
:1065900006E2AEEC37F093EC46F0E552E55201012D
:1065A000C3A1BCDA03DBE552D2D239EC37F0DF6AA3
:1065B00051DBEF6AE6EC37F002E1848906D0E6ECC5
:1065C00036F02C0804E0C9EC37F0000E28D0CCDA05
:1065D00004E1010E4F1801E1B86B0D0EFCEC37F031
:1065E00009E02C0E4F6EF2DB4F5C04E0FC0EDB503A
:1065F000DF5C02E3DF5013D0E9DBE66E2BDBE55214
:10660000E750EF6EB1DA04E1010E4F1801E1B86B0B
:10661000DF2AFD0EDB2AFE0EE0E3DB2ADED7E552A1
:1066200096D290DA090EE126080EDB6AE6EC37F026
:1066300005E1FB0EDB501AE1848918D0C7DB2C087A
:1066400007E0FB0EDB5002E1C9EC37F0020E1AD175
:106650008BDA04E1010E4F1801E1B86B0D0EFCEC72
:1066600037F006E1FB0EDB5001E18489030E0AD10D
:106670002D0EFCEC37F020E1040E4ADB1DE0050E88
:10668000506EFE0EDB50505C17E0FE0EDB0401E1A5
:10669000C0D0030E28DB01E1BCD0070E39DB01E1DD
:1066A000B8D0010EF36E080EF3CFDBFF5DDA04E124
:1066B000010E4F1801E1B86B040E15DB09E0050E61
:1066C00027DB06E00A0EEADAE6D8E2EC37F031D052
:1066D00000EC38F0EFCF4EF0000E4EC0DFFF45DB90
:1066E000050E01DB1FE1000EDFCFE6FF010EDBCF61
:1066F000E6FF2AEC4CF0E552E552F3CF4EF0F4CF32
:106700004FF0506A516A4FAE02D0506851684EC087
:10671000DFFF010E4FC0DBFF020E50C0DBFF030E98
:1067200051C0DBFF040120DA04E1010E4F1801E142
:10673000B86B080EDB5040E0FE0EDB5006E14DDA90
:10674000800E6ADA000EEE5412E3020ECCDA06E195
:1067500044DA000EEE54800E5FDA09E3060ED8DA52
:1067600008E13BDA000E58DA800EEE5402E2040132
:1067700050D077DA080EDB5053E0040EDBCF40F048
:10678000050EDBCF41F0060EDBCF42F0070EDBCF6C
:1067900043F0456846684768486871EC4BF0040E62
:1067A0003CC0DBFF050E3DC0DBFF060E3EC0DBFF3D
:1067B000070E3FC0DBFF34D0FE0EDB5006E10DDAE2
:1067C0007F0EEE54000E28DA23E3FE0EDB0404E114
:1067D00071DB000E21DA1CE3020E85DA04E16ADBCC
:1067E0007F0E1ADA15E3030E93DA04E163DBFF0E82
:1067F00013DA0EE3060E506EFE0EDB50505C0CE119
:1068000059DBFF0EEE54FF0EEE547F0EEE5404E201
:106810000401848D010E36D0070E65DA01E021DA1D
:10682000FE0EDB50070A21E0010A17E0050A11E01D
:10683000010A0FE0030A08E0050A06E0010A04E085
:10684000050A02E0040E1ED022DA040EDBCFEFFFB1
:1068500018D074DBDBCFEDFF14D070DBDBCFEEFFA5
:10686000060EDBCFEEFF070E0AD011DADFCFEEFF08
:10687000010EDBCFEEFF020EDBCFEEFF030EDBCF10
:10688000EEFF000E4E6E090EE15C02E2E16AE55297
:10689000E16E4E505CD1A0DBDDD9EE6AEE6AEE6AA5
:1068A000EE6A010EDB6AFC0EDB50F36E010E16DAA7
:1068B0004EE20401A5DBEFCFDFFF300EDF5C42E3E9
:1068C000DF5039083FE3C6D9EECF4EF0EECF4FF0A0
:1068D000EECF50F0EFCF51F00A0E456E466A476A90
:1068E000486A4EC040F04FC041F050C042F051C025
:1068F00043F071EC4BF03CC04EF03DC04FF03EC059
:1069000050F03FC051F0300EDF5C526E536A546A53
:10691000556AE8504E2653504F225450502255503D
:10692000512298D94EC0EEFF4FC0EEFF50C0EEFF8F
:1069300051C0EEFF040118D907E1010E4F1804E120
:10694000B86B02D0000E04D0010EDB2AACD7010ECA
:106950004E6E020EE15C02E2E16AE552E16E4E50DB
:10696000F6D05A0E4E6E8B0ECFD87EC44EF0BDDAE6
:10697000FCEF36F00501BC5108E0010E4E6E65508B
:10698000020B01E0010E4E5C17E1CDD90BE1ED5198
:10699000EE1111E18C86A00EED6F0F0EEE6F010E61
:1069A000EF6F1200ED51EE1152E18C96A00EED6FDB
:1069B0000F0EEE6FEF6B1200BC0509E0020EBC5D1E
:1069C00006E0040EBC5D03E0100EBC5D17E1ABD920
:1069D0000BE1ED51EE1111E18C86200EED6F4E0EA4
:1069E000EE6F010EEF6F1200ED51EE1130E18C965B
:1069F000200EED6F4E0EEE6FEF6B1200200EBC5DA1
:106A000026E191D907E1ED51EE1121E18C86D5D92E
:106A1000010E15D0EF0507E1ED51EE1118E18C964E
:106A2000CCD9020E0CD0020EEF5D0BE1ED51EE1150
:106A30000EE18C86A00EED6F860EEE6F030EEF6FEB
:106A40001200ED51EE1103E18C96B7D9EF6B1200F5
:106A500079D8A7D9E8AE02D04E3403D0E750D88019
:106A60004E5423E3FD0EDB5010E00CD9F6BEF76860
:106A7000AAD804E0E846FE0B4F06FCE14E6E02D9B0
:106A8000F6BEF768F9D9EF1210D0FCD8F6BEF76859
:106A90009AD804E0E846FE0B4F06FCE1E81C4E6E77
:106AA000F1D8F6BEF768E8D9EF1651D04BD879D9AE
:106AB000E8AE02D04E3403D0E750D8804E5423E3E2
:106AC000FD0EDB5011E1DED8F6BEF7687CD804E09D
:106AD000E846FE0B4F06FCE1E81C4E6ED3D8F6BE2E
:106AE000F768D2D9EF160FD0CDD8F6BEF7686BD8BD
:106AF00004E0E846FE0B4F06FCE14E6EC3D8F6BE3E
:106B0000F768C2D9EF1223D0A4D9E2EF37F0E66ECE
:106B100088DDF9EF36F061D9D1EF37F0010EA4EF3F
:106B200037F0EA6A000FE96E030EEA2212007AD902
:106B3000E66AA9EF37F09951E96EEA6AD890E9362A
:106B4000EA361200D9CFE6FFE1CFD9FF1200E552B5
:106B5000E7CFD9FF120048DA40D985EF37F0E66E6B
:106B6000000EDA20E66E1200B82BB8514E6E4F6A56
:106B7000000E4E181200E96EDACFEAFFEECFE6FF04
:106B8000EECFE6FFEECFE6FFEFCFE6FF1200E66EB8
:106B900083EC26F0E5521200D890F336E806120096
:106BA000EA22EECF56F0EFCF57F01200E66A0FEC74
:106BB0002AF0E5521200010EF36EDB5012004E6E09
:106BC000DF504E5C1200270EF626950EF7220800C5
:106BD000F5504F6E010E4F521200D9CFE9FFDACFB8
:106BE000EAFFD8801200BAD9100EE66E97EF37F0A0
:106BF000DF50EA6AD50FE96E040EEA221200F7228E
:106C00000900F5CFE9FF0800F5CFEAFF4E5012006A
:106C10004E6E6BD9E66E1200EE54000EEE54000E6E
:106C2000EE541200DF6EDFCFE6FFB6514F6A000F61
:106C30004E6E020E4F224EC0E6FF4FC0E6FFECEC58
:106C400043F0E2EF37F0E76E010EE7CFDBFF040120
:106C500084511200FD0EDBCFE9FFFE0EDBCFEAFF11
:106C60001200D9CFE9FFDACFEAFF040EEECFDBFF47
:106C7000050EEECFDBFF060EEECFDBFF070EEECFED
:106C8000DBFF1200FE0EDBCFF6FFF76A1200FC0EF0
:106C9000DBCFE9FFFD0EDBCFEAFF1200E66EA9EFC6
:106CA00037F09951EA6A710FE96E000EEA22EF504F
:106CB0000001EA6A9C25E96E9D51EA221200010E4C
:106CC000E66EE66A12EF37F0DECF4EF0DDCF4FF022
:106CD0001200DECFE9FFDDCFEAFF1200DBCFF4FFC9
:106CE000F350F45C12004E6EFE0EDB504E5C120050
:106CF0004F22DF50E8244E24E96E000E4F20EA6E4A
:106D0000E552E750EF6E1200DBCF4EF075EF37F033
:106D10004F6EFE0EDB504F5C1200C7C4E6FF83ECE3
:106D200026F0E55212000401ED07000EEE5BEF5174
:106D300012004E6E080EE15E4E501200030EDB5044
:106D4000EA6A400FE96E020EEA221200EF50E66E88
:106D5000E66A2AEC4CF0E552E5521200010EDBCF58
:106D60004EF0020EDBCF4FF01200010EDB6A020E76
:106D7000DB6A030EDB6A12000401B76BB86B040117
:106D8000010EEB6F1200030EE66ECDC44EF0CEC4C2
:106D90004FF01200FE0EDB50F80F4E6E010E4E52F9
:106DA0001200FE0EDBCF4EF0190EE76E4E181200E9
:106DB000EA22EF6ADF2A010E1200100EED6F270E95
:106DC000EE6F1200CCDE010E87EF35F019D9EF50CF
:106DD0001200E6DEEAD8EA2212004FC0E6FF50C0F9
:106DE000E6FF51C0E6FF1200E126E66AE66A97EF89
:106DF00035F0E8D8E55212004EC0E6FF8CDE8EEF8B
:106E000035F0010E4BDF83DE23EF36F0F2D82C0E87
:106E1000C7EF35F079DE8EEF35F08DDE890EE9268D
:106E2000000E1200F1EC29F0E552E5521200D950A3
:106E3000060FA1DE9FEC46F04E6E050EE15E4E5051
:106E40008EEF35F0D890E936EA36000EE926010ECD
:106E500012004F6E506A4EC0E6FFE66E50C0E6FF6D
:106E600082EF46F094DE270E92DE58DE0401848B1A
:106E7000120068DEE6521200D890F636F736F50EAC
:106E8000F626940EFFEF35F0D890F636F736C30E9F
:106E9000F626940EFFEF35F0010EE66EE66E97EFE4
:106EA00035F0940E4E6E8B0E84EF35F00401B75121
:106EB00091EF35F092DEFF0EEE54120076D8D0EF4F
:106EC00035F0CF0E4E6E8B0E1FDE8DEF36F03A0E84
:106ED0005EDE020EE66EC7C44EF01200DBCFE6FFA8
:106EE00083EC26F0E5528EEF35F04F6A506A516A16
:106EF0001200EADE400E4E5C000E4F581200040EE7
:106F0000DB500FDEEF502C0812009FEC46F0526E63
:106F1000050EE15E52501200D7DE000E4E5C100EE0
:106F20004F58120060DEEFEC4AF099EF36F0E66A57
:106F3000E66AF80EE66EE66AE66A1200A8DE040E5D
:106F4000DBCFEEFF050E1200E66E0FEC2AF0E552E5
:106F50001200D9CFE6FFDACFE6FF1200D50EE66EBB
:106F6000040EE66E1200D3DDE66AD9501200010F5E
:106F700029DFE66AD950020FE2EF36F0DCDD790E48
:106F8000E926000EE9EF36F04EC0E6FF26DF13EFEC
:106F900038F0620E4E6E8B0EB7DD040117DF32EF54
:106FA00037F0D9EC46F0F9EF36F0C5DD610EE92691
:106FB000000E1200C7DD030EF4EF36F0C3DD030E42
:106FC000E1261200E552E552E55212000D0E4E6E1A
:106FD0000401FCDE4E5C1200B5DD020EE12612005B
:106FE000E66AE66A12EF37F0506A516A4EC0E6FF71
:106FF00012000EDE8BEF35F04E6EE8DE4E5C1200B6
:10700000B85191EF35F0D6DF050EADDFB0DF0401EA
:1070100084511200D7DE04018451120093DD020E68
:10702000E3DE010E1200F5EC46F0E3DE8EEF35F004
:1070300082EC3EF0A098636A626A0F01266B61ECF5
:107040003EF00F0120EC3EF0DF6ADF504E6E4F6ADB
:107050000C0E4E5C000E4F5810E2DF50040DF3CFC3
:10706000E9FFF4CFEAFF000EE926040EEA22EE6AF9
:10707000EE6AEE6AEE6ADF2AE8D7658C0F01386B9C
:107080006598659C62A607D062960501D36BD86BA4
:10709000D96BDA6BF7D70501010EEC6FED6FEE6B74
:1070A000EF6BE06BDF6A030EDF5C11E2EA6ADF344C
:1070B00085EC3EF0EA22EE6AED6AEA6ADF348CEC97
:1070C0003EF0EA22EE6AED6AE1EC3DF0ECD7050114
:1070D000080EC96F040ECA6F0F01160E266F040149
:1070E000300E026F040E036F400E016F840E006FAE
:1070F0000501BD6BBC6BE552B3EF3DF082EC3EF099
:1071000082BE06D0656A0F01366B0501BC6B6FD07D
:107110000501BC510CE1656A0F01366B20EC3EF0B5
:1071200065B602D06586FCD70501010EBC6FBC05B3
:107130000AE165BA08D0626A0F01366B368136897A
:107140000501020EBC6F6250040B06E00F013651C0
:10715000040B02E0629447DB65B249D06250010B38
:1071600009E00F013651010B05E062DF0501040E55
:10717000BC6F62906250100B06E00F013651100B8D
:1071800002E026DB629862AC10D00F0136AD05D06C
:1071900027EC3EF0730EA0EC3DF0629C0501EA5135
:1071A00001E0EA07EA5101E1F4D86250200B05E062
:1071B0000F013651200B01E0FADA6250020B0CE0AD
:1071C0000F013651020B08E027EC3EF0E6687F0E17
:1071D000E66E93EC3EF0636A040E0501E76EBC199F
:1071E000E8AE02D0E73402D0E750BC5D02E2A198DD
:1071F0002FD00F0136A72BD0DF6A040EDF5C27E209
:1072000062A625D064CFE1F50501E151780BE84293
:10721000E842E842E26F6296E1B504D0E2519AECAE
:107220003EF003D0E2519FEC3EF0EA22EF70E251D3
:1072300002E1E6DA0AD0000EE66EE66AE10EE66EDC
:10724000050EE66E720EA0EC3DF0DF2AD6D7A198AF
:10725000E552B3EF3DF053EC3EF0FD0EDBA403D05E
:10726000E66A18EC3EF0FD0EDBA204D0010EE66EDD
:1072700018EC3EF0FE0EDB504F6A260F4E6E0F0EDE
:1072800012EC3EF0A4EC3DF0FD0EDBCFEFFF020E62
:10729000E15C02E2E16AE552E16EB3EF3DF053ECEE
:1072A0003EF0FD0EDB5003E09BEC3DF002D0D2EC53
:1072B0003DF0FEEC3DF0D9CFE9FFDACFEAFFEE502A
:1072C000ED1003E1F36AF46A28D0A4EC3DF0AEECD3
:1072D0003EF0FB0EDBCFEEFFFC0EDBCFEDFFA4ECB0
:1072E0003DF0EE52FA0EDBCFEFFF400EA4EC3EF085
:1072F000880EB3EC3EF0FD0EDB5003E09BEC3DF05E
:1073000002D0D2EC3DF0EA22EF74DECF4EF0DDCFBA
:107310004FF04EC0F3FF4FC0F4FF020EE15C02E2FB
:10732000E16AE552E16EB3EF3DF053EC3EF0FE0E44
:10733000DB5003E16AEC3EF009D0D7EC3DF041ECC4
:107340003EF0D7EC3DF0010F41EC3EF0020EE15C67
:1073500002E2E16AE552E16EB3EF3DF0AEEC3DF0E2
:1073600065A816D07BEC3EF0400EEE16EE6AEE6A93
:10737000EE6A7BEC3EF0EE7CDEDBEA22EF74400E40
:107380004E6E7BEC3EF04E50EF167BEC3EF0EF7C09
:10739000EAD30501EC5122E1010EEC6FED511EE143
:1073A000010EED6F020ED05D07E1D3DBEE52EF6A06
:1073B000D0DBC80EEF6E1200D00510E1E36BDFDB0F
:1073C000EE52400EEF6EDBDB4DEC3EF0D8DB840E70
:1073D000EF6E010EE36FABDB800EEF6E1200050166
:1073E000EE6BEF6B020ED05D06E1A8EC3EF0CCDB5D
:1073F0003CEC3EF010D0D4510401365D0501D5516E
:107400000401375904E236C4D4F537C4D5F561D840
:10741000A0DBBADB9EDBC80EEF6E120053EC3EF031
:10742000000EDE6E040EDD6EC2DB040DF4CF4FF0F5
:10743000D9CFE9FFDACFEAFFF350EE264F50ED2225
:1074400083DBEF9EFD0EDB5002E1ACDB01D073DB92
:10745000EA22DECFEEFFDDCFEDFF76DBEF9C74DBC3
:10746000040EE926000EEA22EF8C020EE15C02E235
:10747000E16AE552E16E77D365980501D3BF0DD07F
:10748000D8AF09D0020ED06FEF5101E1A8DF05019E
:10749000ED6BEC6B12006AEF3EF0040130AF0DD0E3
:1074A0000501010ED06FEE5101E199DF0501ED6B91
:1074B000EC6BEB510DE1C9EF39F00501020ED06F15
:1074C00036DB840EEF6EED6BEC6BEB5101E161DFAF
:1074D000120082EC3EF0400EDF6E0501D45D000E1E
:1074E000D5590AE2D4C5DFFFCF5102E1010E03D026
:1074F000CF0502E1020ECF6FDF504F6AE850D45D36
:10750000D46F4F50D559D56F24DBEE52DFCFEFFF4C
:10751000380EDD6F040EDE6FD3B10DD0DF5017E0F3
:10752000D1C5F6FFD2C5F7FFD12B000ED22308003C
:10753000F55057DBF3D7DF500AE0D1C5E9FFD2C5DC
:10754000EAFFD12B000ED223EF504BDBF4D7E552EC
:107550000AD3A9DB14DBEE52EFCFDFFFDFCF4EF013
:107560004E500501D95D000EDA5902E2D9C5DFFFA0
:10757000DF504E6E4F6AE850D95DD96F4F50DA59DF
:10758000DA6F010EDB6ADF50F36E010EDBCFF4FF22
:10759000F350F45C16E2010EDB50EA6A380FE96E34
:1075A000040EEA22EF50E66ED6C5E9FFD7C5EAFF22
:1075B000D62B000ED723E552E750EF6E010EDB2AE3
:1075C000E2D7000ED880D955000EDA550DE2C0DBA7
:1075D000DBDAD5DAEF50400B03E14EDBC80E02D008
:1075E0004BDB880EEF6E12D0A2DA840EEF6EDB5109
:1075F000DC1107E005D0DCC5FAFF0501DB51F96EAF
:10760000FADF0501D89FEB5101E1C3DE020EE15C18
:1076100002E2E16AE552E16EA6D274DB0501D38F86
:1076200050DB300EE66EE66AE66A000EE66E040E89
:10763000B1DA658CDF6A030EDF5C02E2C2DAFBD7E7
:10764000010EE66EE66AE66ABE0EE66E050EA2DA88
:10765000659C0501080EC96F040ECA6F000EBF6F4E
:10766000040EC06FBFC5C1F5C26F32C4BDF5BD51B8
:1076700002E1100E0BD0010EE66EE66ABD0EE66E5C
:10768000050EE66E010E5CDA0501200EBC6FE552B8
:107690006AD2800E0401305D4EE10501C00ED36F49
:1076A00004013351030A25E0010A09E0030A41E11C
:1076B0000501520ED16F970ED26F120E34D0325197
:1076C000F66EF76AD890F636F736A70EF626970EBE
:1076D000F7220900F5CFD1F50A00F5CFD2F5020E59
:1076E0000501BCDAF5CFD4F5030EB8DAF5CFD5F540
:1076F0001200040E325D1AE20501D38104013251F9
:10770000E96EEA6AD890E936EA36F60EE926020E04
:10771000EA22EECFD1F5EDCFD2F5D1C5E9FFD2C542
:10772000EAFFEF500501D46FD56B12000501D36B52
:1077300012000501D36B1200B6DA0401386B396B05
:1077400030511F0B020A11E0030A0CE0010A1EE18E
:107750000501D38F040138810501DF0517E104011C
:10776000388314D00501D38F11D00501D38F0401C4
:1077700034BF02D0B6DA01D0B9DA40DABFDA06E0B7
:10778000E3D9EF50040B02E0010E386F0501D3AFCF
:1077900007D0380ED16F040ED26FD381020ED46F92
:1077A000020EE15C02E2E16AE552E16EDCD10F011A
:1077B00026A10CD0E4D9EF50800807E1CAD9EF50D8
:1077C000840803E1DCD98C0EEF6E2691629A1200D8
:1077D0000F013685629865820501010EE06F14DAAB
:1077E000750EA0EF3DF00501E06B0EDA740EA8D91E
:1077F00065920F01369562A402D06294FCD7120004
:1078000081DA05012D0EEA6FFD0EE11539E17E0EDC
:10781000E115E8407F0B040DF3CFBFF5F4CFC0F5C1
:10782000000EBF27040EC023BFC5C1F5C0C5C2F5F9
:10783000C175A5D9EF503C0BE842E8420D081EE1A6
:10784000DF6A080EDF5C16E29AD9020EE926000E06
:10785000C2D9EF50E66EDF50EA6A300FE96E040ECF
:10786000EA22E552E750EF6E8AD978DAEE2AEF2263
:10787000DF2AE7D784D911DA0AD807D023D805D070
:10788000FD0EE115040801E12CD8E5526CD105018B
:10789000CF6BEB6BEE6BEF6BE36BD06B5AD9EF9E5C
:1078A000C97557D9EF9EC975E7D9EF9ED36BD46BD5
:1078B000D56BD86BD96BDA6B51D8A6D9030E40D9EA
:1078C0003CEF3AF0020E0501D05D02E1A9EF3AF07B
:1078D000D06BE35104E12BD98C0EEF6E1200E36BF9
:1078E000120010DA36D9EF50400B01E0010EDF6EC6
:1078F0000501C975080EBC5D0BE132C438FF0F01EC
:10790000385103E00501100E02D00501040EBC6FD2
:10791000D00513E11ED938D9DCDD020E0501CF5D9B
:1079200003E117D9840E07D0DF5003E112D9C80E46
:1079300002D00FD9880EEF6E0FD0D8AF0CD0DB512C
:10794000DC1107E005D0DCC5FAFF0501DB51F96E5B
:10795000FADF0501D89FD06BE55205D10401305103
:10796000600BE842E842E842E842E842000901E0F0
:10797000120031510C0A45E00B0A3FE00C0A31E0DD
:10798000010A22E00B0A1EE0020A1CE0030A18E0CA
:10799000080A10E0010A0CE00F0A08E0030A01E0FF
:1079A00012000501D38F080EBC6F120049EF3BF0A7
:1079B0000DEF3BF00501BD0ED16F050ED26F0CD05F
:1079C0009CEF3BF002EF3DF034510501D16FD26BDB
:1079D000BE0ED127050ED223D381010ED46FD38FD3
:1079E00012000501D38F04013451EA6ABE0FE96E1B
:1079F000050EEA2232C4EFFF120006D9020EA0EFF4
:107A00003DF01200ABD8050EE1260401320510E16D
:107A100030511F0B00090CE10501D38F030E040147
:107A2000315D04E10501010EDF6F02D00501DF6B5E
:107A30000401325101E074D030511F0B020870E193
:107A400034510F0B00096CE034510F0B020868E34E
:107A5000200E0501BC5D64E1D38F040134BF04D066
:107A600040D9CCD8D7D803D041D9C8D8D7D8EA2262
:107A7000020EEFCFDBFFF9D8010B03E1000EDF941C
:107A800001D0DF8434BF02D02CD901D02FD9EA2213
:107A9000DECFEEFFDDCFEDFF030E315D0CE12ED921
:107AA00007E034BF02D0B6D801D0B8D8EA22EF82BE
:107AB000840E59D935D0DF7421D906E045D8EF9E20
:107AC00043D8EF8CF4D802D03FD8EF8CDF74CDD8F8
:107AD000020B02E113D90DE0040134BF02D09AD8A1
:107AE00001D09CD8EA22EF923B0E4E6E2DD9DFD802
:107AF00002D03B0E29D9040134510F0B4F6A260FD7
:107B00004E6E0F0E4F22030E4EC0DBFF040E4FC011
:107B1000DBFF030EDBCFE9FF040EDBCFEAFFEF90C4
:107B2000050EE15C02E2E16AE552E16E1CD010D97B
:107B3000B4D83CEF3EF0FE0EEA6ADB3485EF3EF04F
:107B4000E66EE66A93EF3EF0DECFE9FFDDCFEAFFB7
:107B50001200C9C5E9FFCAC5EAFF1200D9CFE6FF86
:107B6000E1CFD9FF1200E552E7CFD9FF120034511F
:107B70000F0BE96EEA6AD890E936EA361200BFC503
:107B8000E9FFC0C5EAFF1200E9D8380EEE6E040E18
:107B9000ED6E1200E66EF9EC4BF04E6E050EE15EF6
:107BA0004E501200FE0EEA6ADB348CEF3EF0FD0E02
:107BB000DB50E824506EFE0EDB50040DF3505024D1
:107BC0001200DF50BCD8EA22EF6ADF50B3D8EA22B5
:107BD000EF6ADF2A1200EA22EE50EFCFEAFFE96EE9
:107BE0001200E66EDDC5E9FFDEC5EAFFDD2B000E03
:107BF000DE23E552E750EF6EDF061200EA22EECFF9
:107C0000DEFFEDCFDDFF1200000EE66EE66AE66EE7
:107C1000E66A120034510F0B9AEF3EF034510F0B0D
:107C20009FEF3EF04F224EC0DEFF4FC0DDFF12003F
:107C3000FE0EDBCFE6FF0EEC3AF0E552E552120005
:107C4000160E396F9F0E376F7B0E366F1200010EC6
:107C5000E66EE66A000EE66EE66A1200F76AD12565
:107C6000F66ED251F72208001200D950020FE96EC9
:107C7000DACFEAFFEF501200C1C5E9FFC2C5EAFF43
:107C80001200040DF3CF4EF0F4CF4FF0000E4E264D
:107C9000040EC8DF840EB3EF3EF060D8300EEE6EF7
:107CA000040EED6E12005ADF020EE1261200020EE3
:107CB000E66EE66ADECFE6FFDDCFE6FF050EA0EF5B
:107CC0003DF0020EE66EE66AE66A270EE66E0F0EDD
:107CD000CAEF3DF02CDF8C0EEF6E3BDF840EEF6EB3
:107CE000120045DFC30EE926050E120040DFC90E63
:107CF000E926050E12001FDFEBEF3DF025DFEF5008
:107D0000800B12002BDFE6521200FE0BEA36E96E02
:107D1000C90EE926050E1200FE0BEA36E96EC30E07
:107D2000E926050E1200E6EC48F04E6E060EE15E06
:107D30004E501200EA6AE70FE96E050E1200EA6A79
:107D4000E40FE96E050E1200FFDEE850EF16120098
:107D500093DFEE52400EEF6E3CEF3EF0020EE9264E
:0E7D6000000EEA221200F0DEE850EF121200D0
:027D6E00F6D944
:107D7000E6520001606B996BDF6A080EDF5C13E26C
:107D8000E7D9610EE926000E12DAC8D9EF6AE0D908
:107D9000790EE926000E0BDADBD9890EE926000EF2
:107DA00006DADF2AEAD70001C60E9C6F0E0E9D6F21
:107DB0003F0E79140009796ECF0E79140009796E9F
:107DC00079827B6A7A6A79900F0152815293F00E20
:107DD000B4140909B46E0001080E9A6F030E9B6F6C
:107DE000C60E9E6F3B0E9F6F250EA06F580EA16FA3
:107DF000040EA66F900EA26F010EA36F900EA46FDB
:107E0000010EA56F000EE66EE66A010EE66E7DECD1
:107E100016F0E552E552E5528996E552A4D19ED975
:107E2000E652DF6A080EDF5C09E278D9EFCF4EF048
:107E3000FE0EDB504E5C09E0DF2AF4D7DF6A080E45
:107E4000DF5C07E26BD9EF5002E1DF2803D0DF2AC5
:107E5000F6D7000EE55287D181D9070EE126DE6AFA
:107E6000DD6A020EDB6A030EDB6A040EDB6A050EB6
:107E7000DB6A060EDB6A010EE66ED9CFE6FFDACFCB
:107E8000E6FF030E39D9020F7AD9010E35D9030F57
:107E900076D9030E31D9050F72D9030E80D9E66A5F
:107EA000E66AF1EC29F0E552E5520401845124E13F
:107EB000020EDB50180802E2848D1ED0010EE66E21
:107EC000050EDBCFE6FF060EDBCFE6FF030EDBCFB2
:107ED000E6FF040EDBCFE6FF020EDBCFE6FFDECFD0
:107EE000E6FFDDCFE6FF0FD84E6E080EE15E4E5086
:107EF000E66A0FEC2AF0E552070EE15C02E2E16A65
:107F0000E552E16E30D12AD9020EE126FC0EDBCF1C
:107F1000E6FF85DFE552E76E010EE7CFDBFFDB50C2
:107F200002E1000EC3D00BD902E1C9D8BDD0010EC9
:107F3000DB044E6E00019A514E5C01E3B5D0FC0E9D
:107F4000DB50180801E2B0D0FC0EDB50070802E15C
:107F50000101C16BD6D810E1E66AFC0EDBCFE6FF6B
:107F600056EC35F0E552E552E66AFC0EDBCFE6FF53
:107F700028EC35F0E552E552F70EDB046AE11350C8
:107F80000F5CFDE2FC0EDB50040801E1C9D809BC1E
:107F90008BD0D0D8020EEF6EF80EDBCF4EF0F90E7C
:107FA000DBCF4FF0506A516A190E456E466A476A38
:107FB000486A4EC040F04FC041F050C042F051C03E
:107FC00043F071EC4BF03CC04EF03DC04FF03EC072
:107FD00050F03FC051F0AED8EE52EE523CC0EEFF32
:107FE0004FC0EEFF50C0EEFF51C0EEFF80D8290E0B
:107FF000E926000EEA22010EDBCFEFFF78D8260E2D
:10800000E926000EEA22FC0EDBCFEFFF70D8270E28
:10801000E926000E7BD86BD82A0EE926000EA7D8D9
:1080200066D8EE52D880000EEE54000EEE54190EB3
:10803000EE54000EEE5406E25AD8EE52EE6AEE6AA4
:10804000EE6AEE6A102A1350105C01E3106A0F2AE0
:108050002BD005A029D0FC0EDB50040801E160D82C
:108060006ED802E12CD812D08FD8890EE926000EE6
:108070007ED88AD8790EE926000E48D88DD8FC0E15
:10808000DBCFEFFF3ED802E19DD840D8FC0EDB509D
:108090000001A65D09E10101010EB96F0101B66B96
:1080A0000101C15101E08A98010EDB504E6E020EB3
:1080B000E15C02E2E16AE552E16E4E5054D06CD8C8
:1080C000EF500001EA6A9C25E96E9D51EA22EF6AB1
:1080D0005BD8890EE926000E6AD856D8790EE926B3
:1080E000000E65D859D8EF6A6DD8D7EF40F0105020
:1080F0002F0D61D8EE52120052D8010EE66ED95003
:10810000120060D8EA22EE50ED101200EA22FD0EB5
:10811000DBCFEEFFFE0EDBCFEDFF1200DF5057D0BE
:108120008986C2C4BEF4C3C4BFF4C4C4C0F4C5C409
:10813000C1F4120010502F0D0501DBEF40F0D950B3
:10814000FD0FE96EFF0EDA20EA6EEE50ED10120020
:10815000EA6ADF34FE0BEA36E96E1200D9CFE6FF99
:10816000E1CFD9FF1200E552E7CFD9FF1200EA2292
:10817000FA0EDBCFEEFFFB0EDBCFEDFF1200E66E5B
:10818000000EDA20E66E1200010EDB04E96EEA6AE8
:10819000D890E936EA361200010EDB0418D0E66EFC
:1081A00011EC33F0E552E552E552E5521200EA22B5
:1081B000EE6AED6A1200FA51F324E96EFB51F420E5
:1081C000EA6E1200E1DF610EE926000E1200EA6A93
:0A81D000710FE96E000EEA221200A2
:0681DA003B9E0CD03B9E11
:1081E00043AE09D0406C411E421E431EE86A412244
:1081F000422243223B8E43C03DF042C03CF041C08E
:108200004DF040C04CF09E0E3E6E3F6AB6EF42F01D
:108210003B6AF2EC42F00AEC43F03BB69AEF42F0D4
:108220003BA205D03BBA9AEF42F0A1EF42F03BBA35
:10823000ADEF42F03BA005D03BB89AEF42F0ADEF76
:1082400042F03BB8A1EF42F03F6A7F0E44243E6EFD
:10825000E86A3F2249503E5EE86A3F5A1A0E4A6E6B
:10826000446A4C6A4D6A3C6A3D6A4650415E4750DA
:10827000425A4850435A000E445A09E74650412694
:108280004750422248504322000E442201D04C8ADB
:10829000D8904136423643364436D8904C364D3627
:1082A0003C363D364A2EE1D7435042104110D8A407
:1082B0004C8AB6EF42F03B6AF2EC42F00AEC43F033
:1082C0003BB69AEF42F03BA205D03BB89AEF42F0A2
:1082D000A1EF42F03BAA05D03BB09AEF42F0A1EFEC
:1082E00042F03BB002D03BA802D0ADEF42F03F6A73
:1082F000495044243E6EE86A3F227E0E3E5EE86AA4
:108300003F5A4C6A4D6A3C6A3D6A48504302F4CF7A
:108310003DF0F3CF3CF047504302F3504D26F4506C
:108320003C22000E3D2248504202F3504D26F450AC
:108330003C22000E3D2246504302F3504C26F4509E
:108340004D22000E3C223D2247504202F3504C2663
:10835000F4504D22000E3C223D2248504102F35081
:108360004C26F4504D22000E3C223D224650420243
:10837000F4504C26000E4D223C223D224750410233
:10838000F4504C26000E4D223C223D22B6EF42F026
:108390003A6AE86A48AED5EF41F0456C461E471E82
:1083A000481E4622472248223A1E43AEE0EF41F0E3
:1083B000406C411E421E431E4122422243223A1E6D
:1083C000D5EC4BF043BEF7EF41F03AAE000C406CF9
:1083D000411E421E431EE86A4122422243223C6C57
:1083E0003D1E3E1E3F1E3D223E223F22000C3ABE55
:1083F000E7EF41F03B88FF0C3B6AF2EC42F03BB602
:1084000006EF42F03BA20FD03BB407D07F0E436E85
:10841000FF0E426E416E406E25D0800E436E01D03D
:10842000436A000EF6D73BB0FBD7406A9F0E44600C
:10843000EBD77E0E4464F4D79E0E445C07E0D890E0
:108440004332423241324032442AF6D73BA40AD06A
:10845000406C411E421E431EE86A412242224322D2
:1084600043AEDED7120045EC42F03BB6000C3BB009
:10847000000C3BB4000C010C45EC42F03BB6000C88
:108480003BB0000C3BA4000C010C3B6AF2EC42F048
:108490000AEC43F03BB612003BAE08D03BA004D040
:1084A0003BA802D03B8012003B9012004950445C34
:1084B0000BE14850435C08E14750425C05E14650FF
:1084C000415C02E13B801200D8A002D03B8E10D06C
:1084D000445049C044F0496E435048C043F0486E90
:1084E000425047C042F0476E415046C041F0466E90
:1084F0004950445C10E0FF0F09E03B903BB403D0CF
:108500003BAE3B8412003BAE3B941200492AD8900C
:108510004832473246324650415E4750425A4850F0
:10852000435A43BEEAD7D890413642364336442EAA
:10853000F8D7C8D77F0E446EFF0E436E426E416E71
:1085400012007F0E3BBEFF0E446E02D07F0E446EC3
:10855000800E436E426A416AF3D73BAE04D0800E70
:10856000446E436AF7D7446A436AF4D73D503C10DF
:108570004D104C10F8E03FBEF0D73DBE0CD03E5041
:108580003F10EBE0D8904C364D363C363D363E063B
:10859000D8A03F06F2D73F50D4E13E28D2E04CAEFF
:1085A00011D07F0E4C1402E14DA00CD04D2AE86A88
:1085B0003C223D2207E3D8803D323C324D323E2AF8
:1085C0003E28BFE03E50C9E04DC041F03CC042F003
:1085D0003D34436E3E30446E4332449E3BBE448E37
:1085E000A0EF42F04336443602E33B843B7E06E193
:1085F0003B80446A436A426A416A1200442803E0AD
:10860000D88043321200D890433202E13B821200FC
:108610003B8612004836493602E33B8C3B7E06E13E
:108620003B88496A486A476A466A1200492803E05B
:10863000D88048321200D8904832EAE13B8A1200D2
:10864000040130511F0B010801E012003051600B92
:10865000E842E842E842E842E842010801E012004C
:10866000345103E0340501E012003151220A31E0B7
:10867000030A24E0010A15E0210A0DE0010A01E0E5
:1086800012000501B40ED16F050ED26F080ED46F23
:10869000D56BD38121D00501B40ED16F050ED26FF9
:1086A0001BD036C4D9F537C4DAF50501940ED66F60
:1086B000050ED76FDB6BDC6BD88F12000501940EB3
:1086C000D16F050ED26F070ED46FD56BC10ED36F6D
:1086D000120032C4AFF50501D38F12000501946B6F
:1086E0004B0E956F966B976B986B996B080E9A6F04
:1086F000A36B1A0EE66E010EE66E2BEC39F0E55216
:10870000E5521E0EE66E020EE66E2BEC39F0E552D7
:10871000E5521CD90501AD6BAE6BA46B120041D9BB
:1087200065D9050E421801E1435002E0000E14D055
:1087300048D90501AB514E1804E1AC514F1801E185
:1087400005D93FD90501AD514E1805E1AE514F187D
:1087500002E1A46BA96B010E29D123D90501A36BFA
:10876000AB51AC1102E1000E05D032D9EF50800BB5
:1087700001E0010E00092DE1FC0EDBCF4EF028D9FF
:10878000EE52EF50D8804E5405E222D9EE52FC0E44
:10879000EFCFDBFFA36BFC0EDB50A35D19E2A3510F
:1087A000EA6A540FE96E050EEA22EF50E66EA35115
:1087B000E76EFD0EDBCFE9FFFE0EDBCFEAFFE750F1
:1087C000E926000EEA22E552E750EF6EA32BE3D72D
:1087D000BDD80501A351EAD0E4D80501A45107E1B1
:1087E000E9D8FC0EDBCFA9F5010EAA6FA46FDED08D
:1087F00004D917E1C0D8DF2AFF0EDF5C0BE0010EC1
:10880000DBCFE9FFDB2A020EDBCFEAFF01E3DB2A45
:10881000EF50F1E1CFD8DFCFA9F50501010EAA6F26
:10882000A46F030EE15C02E2E16AE552E16EBED0A4
:10883000E4D818E1A0D8DF2AFF0EDF5C0CE0010EBF
:10884000DBCFF6FFDB2A020EDBCFF7FF01E3DB2AEB
:108850000800F550F0E1AED8DFCFA9F50501AA6B0D
:10886000010EA46F030EE15C02E2E16AE552E16EE3
:108870009DD097D8020EE1260501AD51AE1102E15F
:10888000000E08D0ADC5E9FFAEC5EAFFEF50800B82
:1088900001E0010E000953E1030EA45D01E1A46BA8
:1088A000A4514DE0020EA45D09E1E66A000EE66EF9
:1088B000E66A59D80501030EA46F41D0A4053FE133
:1088C000400E4E6E4F6AA9514E5C000E4F5803E2A7
:1088D000400EDF6E02D0A9C5DFFFDF50A95DA96F92
:1088E000140EA76F050EA86F010EDFCFDBFFAA5194
:1088F0000BE1010EDB5012E0A5C5F6FFA6C5F7FFA0
:108900000800F55041D8F5D7010EDB5007E0A5C5AA
:10891000E9FFA6C5EAFFEF5037D8F6D70501A95100
:1089200007E1400EDF5C02E1020E01D0030EA46FEE
:10893000DFCFE6FF140EE66E050EE66E14D8020ECB
:10894000E15C02E2E16AE552E16E30D0400EE66E93
:10895000540EE66E050EE66EE66A3FD8F3CFABF531
:10896000F4CFACF51200010EE66E37D8F3CFADF5BB
:10897000F4CFAEF51200DF6A39D8DE5242C0DEFF16
:1089800043C0DDFFDD521200A7C5E9FFA8C5EAFF1D
:10899000EF6EA72B000EA823A52BA623010EDB0646
:1089A0001200D9CFE6FFE1CFD9FF1200E552E7CFA1
:1089B000D9FF1200FD0EDBCFA5F5FE0EDBCFA6F52D
:1089C0001200FB0EDBCF4EF0FC0EDBCF4FF012009F
:1089D000ABC5E9FFACC5EAFF1200020EE66E4FEC34
:1089E00039F04E6E050EE15E4E501200FD0EDBCFEB
:1089F00042F0FE0EDBCF43F01200D3DF030EE12680
:068A00000501A451120063
:0A8A06002130204572723A203C61D5
:108A1000786973323E2073746570207261746520CA
:108A2000746F6F20736C6F772E0021302045727247
:108A30003A203C61786973323E207374657020720D
:108A400061746520746F6F20686967682E0021303B
:108A5000204572723A203C61786973313E2073740C
:108A60006570207261746520746F6F20736C6F770E
:108A70002E002130204572723A203C6178697331B2
:108A80003E2073746570207261746520746F6F206E
:108A9000686967682E00205341323D002053413100
:108AA0003D004475726174696F6E3D002130204550
:108AB00072723A20537465705261746520696E76E3
:108AC000616C69642076616C75652E005261746515
:108AD0003D00434D20636F6D6D616E64206469736A
:108AE00061626C656420696E2074686973206275C8
:108AF000696C640020446972656374696F6E3D003F
:108B00002043656E7465725F593D002043656E7445
:108B100065725F583D0020446573745F593D0020C5
:108B2000446573745F583D00467265713D00205383
:108B3000453D00204A323D002041323D0020533265
:108B40003D002052323D00204A313D002041313D60
:108B5000002053313D0052313D00537461747573F0
:108B60003D002135204572723A204E6565642063D0
:108B70006F6D6D61206E6578742C20666F756E6404
:108B80003A202700506172616D383D00506172617A
:108B90006D373D00506172616D363D00506172610C
:108BA0006D353D00506172616D343D005061726100
:108BB0006D333D00506172616D323D0050617261F4
:108BC0006D313D000D0A000A0D004F4B000A0021D7
:108BD00038204572723A20556E6B6E6F776E206347
:108BE0006F6D6D616E642027002138204572723AE6
:108BF00020436865636B73756D206E6F7420666FBC
:108C0000756E642062757420726571756972656431
:108C10002E002138204572723A20436865636B73D9
:108C2000756D20696E636F72726563742C20657850
:108C300070656374656420004C696D697420737796
:108C400069746368207472696767657265642E2051
:108C5000506F7274423D002137204572723A2045B0
:108C60007874726120706172616D65746572002143
:108C700036204572723A20496E76616C69642070C4
:108C80006172616D657465722076616C7565002135
:108C900034204572723A204D697373696E67207093
:108CA0006172616D657465722873290021332045F6
:108CB00072723A20525820427566666572206F764D
:108CC000657272756E002132204572723A205458D6
:108CD00020427566666572206F76657272756E00E9
:108CE0002131204572723A2043616E2774207374DB
:108CF000657020746861742066617374002130208F
:048D00000020080047
:0C8D0400DDD8D0D80DE0CED8F3D8D9507F
:108D1000FC0FE96EFF0EDA20EA6EEE2A000EEE225C
:108D2000EE22F1D7F7D0CCD8D6D808E0D4D8E2D804
:108D3000FD0EDB2AFE0EF8E3DB2AF6D7EBD0EED8E9
:108D40000F0E4E6E4F6A506AD950BFD8EE504E1675
:108D5000EE504F16EE505016EE504EC0FEF14E50F3
:108D6000090802E3300E01D0370EFE25C8D873D8AB
:108D7000040ED890513250324F324E32E806F9E1AB
:108D8000FB0E4EC0DBFFFC0E4FC0DBFFFD0E50C0E4
:108D9000DBFFFE0E51C0DBFF0101FD07FA0EDB50C9
:108DA00002E0FA0EDB06C0D8CBE1FA0EDB50C8E1D8
:108DB0006CD0B4D85DD897D83CC0FEF1300E01011C
:108DC0003C249DD855D88FD8FB0E40C0DBFFFC0E4D
:108DD00041C0DBFFFD0E42C0DBFFFE0E43C0DBFFE8
:108DE0000101FD07A1D8E6E150D06AD8E1506DD865
:108DF000D890030EEB50000A08E6000EEE5C000E61
:108E0000EE58000EEE58000EEE5815E22D0E72D8F8
:108E10002FD8456846684768486871EC4BF0FB0EF0
:108E20003CC0DBFFFC0E3DC0DBFFFD0E3EC0DBFFA8
:108E3000FE0E3FC0DBFFD95048D8EECFE6FFEECFA5
:108E4000E6FFEECFE6FFEFCFE6FFB3DFE552E552F8
:108E5000E552E5525FD0FB0EDBCF4EF0FC0EDBCFD0
:108E60004FF0FD0EDBCF50F0FE0EDBCF51F01200C5
:108E7000FB0EDBCF40F0FC0EDBCF41F0FD0EDBCF75
:108E800042F0FE0EDBCF43F01200FD2BFD514F6A86
:108E9000F10F4E6E010E4F224EC0E6FF4FC0E6FFAF
:108EA00042DFE552E55236D0FC0EDBCFF6FFFD0E79
:108EB000DBCFF7FFFE0EDBCFF8FF0800F550120006
:108EC000D9CFE6FFE1CFD9FF1200FB0FE96EFF0E0D
:108ED000DA20EA6E1200FD0EDBCFE9FFFE0EDBCFDB
:108EE000EAFFEF5012000A0E456E466A476A486A6A
:108EF000D5EF4BF0E66E83EC26F0E5521200E66EFD
:108F0000FD51EA6AF10FE96E010EEA22E552E750DF
:108F1000EF6E1200E552E7CFD9FF1200D1DF010159
:108F2000FC6B0A0EFD6F120096DF4E504F10501072
:048F300051101200CA
:0C8F3400D9CFE6FFDACFE6FFE1CFD9FF8E
:108F4000E2CFDAFF060EE12402E3E168E652E16EC9
:108F5000DF6A010EDB6AD950FA0FE96EFF0EDA20E4
:108F6000EA6E020EEECFDBFF030EEECFDBFF040E48
:108F7000EECFDBFF050EEECFDBFFD950FA0FE96E27
:108F8000FF0EDA20EA6E060EE76ED890030EEB3283
:108F9000020EEB32010EEB32EF32E706F6E1D9506A
:108FA000FA0FE96EFF0EDA20EA6E060EE76ED89031
:108FB000EF36010EEB36020EEB36030EEB36E7060C
:108FC000F6E1D950FA0FE96EFF0EDA20EA6E400E94
:108FD000EE26000EEE22000EEE22000EEE22FA0E1B
:108FE000DBCF52F0FB0EDBCF53F0FC0EDBCF54F0A7
:108FF000FD0EDBCF55F0D950020FE96E000EDA20DE
:10900000EA6EEE50525C4E6EEE5053584F6EEE507C
:109010005458506EEE505558516E4E50DF6ED95028
:10902000F80FE96EFF0EDA20EA6EEE50ED1065E003
:10903000040EDB50F86E030EDB50F76E020EDB50B1
:10904000F66EDF50DF0600091AE0F60EDBCFE9FF0F
:10905000DB2AF70EDBCFEAFF01E3DB2AEF50F56EE8
:109060000D00F80EDB06DBCF4EF0F90E01E2DB0659
:10907000DBCF4FF04E504F1001E101D0E2D7040E8C
:10908000DB50F86E030EDB50F76E020EDB50F66E0F
:10909000A684F2AE04D0F29EDE52010EDD6E550EB5
:1090A000A76EAA0EA76EA682A694010EDB5003E05F
:1090B000F28E010EDB6A400EDF6E400E4E6E4F6A7E
:1090C000506A516AD950020FE96E000EDA20EA6E3A
:1090D000EE504E26EE504F22EE505022EE505122CE
:1090E000020E4EC0DBFF030E4FC0DBFF040E50C06C
:1090F000DBFF050E51C0DBFF92D7060EE15C02E2FA
:10910000E16AE552E16EE552E5CFDAFFE7CFD9FF3C
:0291100012004B
:0E911200F5EC23F005D87EEC38F022EC25F0C9
:10912000FBD7D9CFE6FFE1CFD9FF020EE1260F0131
:1091300048694969600ED36E9B8C580EDE6E020E34
:10914000DD6EDFCF4EF0DF06010EDBCF4FF001E228
:10915000DB064E504F10F5E1948E67EC24F018ECCE
:1091600038F0020EE15C02E2E16AE552E16EE5529E
:10917000E7CFD9FF1200120012001200120020EFF8
:1091800043F012006EEF43F00501DF051EE105011B
:10919000E0051BE1F1DF65920501E06B0201100EB5
:1091A000FE6F0E0EFF6FFE07000EFF5BFE51FF11FC
:1091B000FAE16584080EFE6F070EFF6FFE07000ED2
:1091C000FF5BFE51FF11FAE165941200D9CFE6FF73
:1091D000E1CFD9FFFD0EDBCF42F0FE0EDBCF43F037
:1091E000050E421801E1435036E0E868421802E1FA
:1091F0007F0E43182FE0030E421801E1435028E090
:10920000020E421801E1435021E0010E421801E133
:1092100043501AE0740E421801E1435013E0750EFA
:10922000421801E143500CE0730E421801E1435033
:1092300005E0720E42180FE143500DD09EDF0BD0B7
:109240009ADF09D099DF07D09DDF05D09ADF03D0E0
:1092500096DF01D093DF010EE552E7CFD9FF120070
:10926000D9CFE6FFE1CFD9FF0501FB0EDBCF00F53B
:10927000FC0EDBCF01F5FD0EDBCF02F5FE0EDBCFE2
:1092800003F5036725D0026723D0126B800E106FA1
:109290000B6F0B510B03F350005DF4500159D8B024
:1092A00008D012C50BF5104310510B1310BF09D095
:1092B000F0D70BC512F5104310510B1310BF01D09E
:1092C000E8D712C5F3FFF46AE552E7CFD9FF1200E1
:1092D000126B136B106B0B6B800E116F0A6F0BC54B
:1092E00005F50AC504F5A3EC49F00C51005D0D51DC
:1092F00001590E5102590F510359D8B00ED0000F29
:1093000012C50BF513C50AF51133103311510A13A9
:1093100010510B13D8B00FD0E2D7000F0BC512F5C8
:109320000AC513F51133103311510A1310510B13E1
:10933000D8B001D0D4D712C5F3FF13C5F4FFE5525E
:10934000E7CFD9FF120005510503F4CF0DF5F3CF98
:109350000CF504510403F4CF0FF5F3CF0EF50551CE
:109360000403F3500D27F4500E23E86A0F23045131
:109370000503F3500D27F4500E23E86A0F23120063
:10938000C00EF36E00EE00F00E0E01D81200EA607F
:1093900002D0EE6AFCD7F350E9601200EE6AFCD707
:1093A000D9CFE6FFDACFE6FFE1CFD9FFE2CFDAFF90
:1093B000E652E652E652E652E652DF6AD950FA0F1A
:1093C000E96EFF0EDA20EA6E010EEECFDBFF020E31
:1093D000EECFDBFF030EEECFDBFF040EEECFDBFFA5
:1093E000F60EDBCF4EF0F70EDBCF4FF0F80EDBCFF3
:1093F00050F0F90EDBCF51F048D84E50EE5C4F5094
:10940000EE585050EE585150EE5833E2030EDB50F8
:10941000F86E020EDB50F76E010EDB50F66EA6847E
:10942000A688F2AE03D0F29E010EDF6E550EA76E37
:10943000AA0EA76EA682DF5001E0F28E4E6A040EDD
:109440004F6E506A516A21D8EE504E26EE504F2290
:10945000EE505022EE505122010E4EC0DBFF020EA4
:109460004FC0DBFF030E50C0DBFF040E51C0DBFF1B
:10947000B7D7050EE15C02E2E16AE552E16EE55222
:10948000E5CFDAFFE7CFD9FF1200D950010FE96E1F
:08949000000EDA20EA6E120062
:089498004542427631335F6169
:1094A0006E645F61626F7665204542204669726D29
:1094B000776172652056657273696F6E20332E3046
:1094C0002E3200920F920F920F930F930F930F93E0
:1094D0000F930F930F930F930F940F940F940F9478
:1094E0000F940F940F940F940F950F950F950F9560
:1094F0000F950F950F890F890F890F8A0F8A0F8A91
:109500000F8A0F8A0F8A0F8A0F8A0F8B0F8B0F8B90
:109510000F8B0F8B0F8B0F8B0F8B0F8C0F8C0F8C78
:109520000F8C0F8C0F8C0F00010500010203040546
:1095300006070001020304050607020304050607E7
:109540002A0EF66E100EF76E000EF86E0501090079
:10955000F550F56F0900F550F66F03E1F56701D09E
:109560003DD00900F550F06F0900F550F16F09008A
:10957000F550F26F09000900F550E96E0900F55049
:10958000EA6E090009000900F550F36F0900F55073
:10959000F46F09000900F6CFF7F5F7CFF8F5F8CF2B
:1095A000F9F5F0C5F6FFF1C5F7FFF2C5F8FF0501C3
:1095B000F35302E1F45307E00900F550EE6EF307B0
:1095C000F8E2F407F9D7F7C5F6FFF8C5F7FFF9C5D4
:0E95D000F8FF0501F507000EF65BBFD712008D
:0295DE00D9CFE3
:1095E000E6FFDACFE6FFE1CFD9FFE2CFDAFFE652BE
:1095F000E652E652E652D9CFE9FFDACFEAFFFA0E99
:10960000DBCFEEFFFB0EDBCFEEFFFC0EDBCFEEFF82
:10961000FD0EDBCFEEFF020EDB50F86E010EDB50CD
:10962000F76EDF50F66EF80EDBCF4EF0DB06F90E6C
:10963000DBCF4FF001E2DB064E504F100DE009008A
:10964000F60EDBCFE9FFDB2AF70EDBCFEAFF01E303
:10965000DB2AF5CFEFFFE7D7040EE15C02E2E16A17
:10966000E552E16EE552E5CFDAFFE7CFD9FF120010
:10967000D9CFE6FFDACFE6FFE1CFD9FFE2CFDAFFBD
:10968000AD6AAC6AFD0EDBB0AD88DBA202D0AD8C5A
:10969000AC8CDBB4AD8EDBA602D0AC8801D0AC8A3A
:1096A000DBB8AD84DBBAAC86DBAC02D09D8A01D0DE
:1096B0009D9ADBAE02D09D8801D09D98FB0EDB50B9
:1096C000B06EFC0EDBCF4FF04FC04EF04F6A4E50E5
:1096D0007F6EAD8AAC8EE552E5CFDAFFE7CFD9FFDA
:0296E000120076
:0E96E20040504502F3CF3CF0F4CF3DF046027D
:1096F000F3503D26000EF4203E6E40504702F350DA
:109700003E26000EF4203F6E40504802F3503F26A4
:1097100041504502F3503D26F4503E22000E3F22B8
:1097200041504602F3503E26F4503F22415047023A
:10973000F3503F2642504502F3503E26F4503F225C
:1097400042504602F3503F2643504502F3503F2615
:02975000120005
:0E9752001201000202000040D80492FD8201C4
:109760000102030109024300020100C032090400A2
:109770000001020201000524001001042402020578
:1097800024060001052401000107058103080002E9
:1097900009040100020A000000070502024000005F
:0997A000070582024000006497F5
:0697AA003F6A3E6A3D6AC1
:1097B0003C6A200EE76ED89040364136423643363A
:1097C0003C363D363E363F3645503C5C46503D5873
:1097D00047503E5848503F5809E345503C5E46507C
:1097E0003D5A47503E5A48503F5A402AE72EE4D748
:0297F000120065
:0E97F200FE0EE3CFE9FFFF0EE3CFEAFFE9CF63
:10980000F3FFEACFF4FFFB0EE35003E1FC0EE3505D
:1098100009E0FB0EE30602E2FC0EE306FD0EE35058
:06982000EE6EF1D712000C
:0A982600D9CFE6FFDACFE6FFE1CF6D
:10983000D9FFE2CFDAFFADAC04D0AD900501FCB3A7
:10984000AD80FD0EDB50AE6EE552E5CFDAFFE7CF1F
:04985000D9FF12002A
:0C985400FF0EE124E96EFF0EE220EA6E38
:10986000EDCFF4FFEFCFF3FFF46607D0600EF364A3
:0C98700004D07B0EF36001D0F39A1200CC
:04987C00D9CFE6FF5B
:10988000DACFE6FFE1CFD9FFE2CFDAFFFD0EDB5002
:0E9890007E6EE552E5CFDAFFE7CFD9FF12007A
:02989E001EEEBC
:1098A00000F02EEE00F0F86A3B9CA0EC4AF068EC69
:0A98B0004CF089EC48F0FBD71200E1
:0698BA00F36AF46AF32AD0
:1098C0000F0B05E0D890F336F436E804FBE1120004
:0298D000120084
:0E98D2000403090418035300630068006D00CE
:1098E00061006C007A004800610075007300380365
:1098F0004500690042006F00740042006F00610083
:10990000720064002C0020002000200020002000B5
:109910002000200020002000200020002000200047
:109920002000200020002203200020002000200032
:109930002000200020002000200020002000200027
:109940002000200020002000800284029C02D4021B
:0299500000060F
:099952000000000001000000000B
:00000001FF
